:100000000C9489070C94AF070C94AF070C94AF07BE
:100010000C94AF070C94AF070C94AF070C94AF0788
:100020000C94AF070C94AF070C9418090C94340986
:100030000C94AF070C94AF070C94AF070C94AF0768
:100040000C94AF070C94AF070C94AF070C94AF0758
:100050000C94AF070C94AF070C94AF070C94AF0748
:100060000C94AF070C94AF070C94AF070C94AF0738
:100070000C94AF070C94AF070C94AF070C94AF0728
:100080000C94AF070C94AF070C94AF070C94AF0718
:100090000C94AF070C94AF070C94AF070C94E836A0
:1000A0000C9425370C9462370C949F370C94AF074F
:1000B0000C94AF070C94AF070C94AF070C94AF07E8
:1000C0000C94AF070C94AF070C94AF070C94AF07D8
:1000D0000C94AF070C94AF070C94AF070C94AF07C8
:1000E0000C94AF070C94AF070C94AF070C94AF07B8
:1000F0000C94AF070C94AF070C94AF070C94AF07A8
:100100000C94AF070C94AF070C94AF070C94AF0797
:100110000C94AF070C94AF070C94AF070C94F43514
:100120000C9431360C946E360C94AB360C94AF07AD
:100130000C94AF070C94AF070C94AF070C94AF0767
:100140000C94AF070C94AF070C94AF070C94AF0757
:100150000C94AF070C94AF070C94AF070C94AF0747
:100160000C94AF070C94AF070C94AF070C94AF0737
:100170000C94AF070C94AF070C94AF070C94AF0727
:100180000C94AF070C94AF070C94AF070C94AF0717
:100190000C94AF070C94AF070C94AF070C94AF0707
:1001A0000C94AF070C94AF070C94AF070C94AF07F7
:1001B0000C94AF070C94AF070C94AF070C94AF07E7
:1001C0000C94AF070C94AF070C94AF070C94AF07D7
:1001D0000C94AF070C94AF070C94AF070C94AF07C7
:1001E0000C94AF070C94AF070C94AF070C94AF07B7
:1001F0000C94AF07ED19EA19E719E419E119DE19B2
:10020000DB19D819D519D219CF19CC19C919C619A2
:10021000C319C019BD19BA19B719B419AE19B11952
:100220003C696E70757420747970653D22737562D7
:100230006D697422207374796C653D226865696705
:1002400068743A203530707822206E616D653D22E9
:10025000746F67676C65222076616C75653D224C12
:10026000454434222F3E266E627370266E62737090
:100270003C696E70757420747970653D2273756287
:100280006D697422207374796C653D2268656967B5
:1002900068743A203530707822206E616D653D2299
:1002A000746F67676C65222076616C75653D224CC2
:1002B000454435222F3E266E627370266E6273703F
:1002C0003C696E70757420747970653D2273756237
:1002D0006D697422207374796C653D226865696765
:1002E00068743A203530707822206E616D653D2249
:1002F000746F67676C65222076616C75653D224C72
:10030000454436222F3E266E627370266E627370ED
:100310003C696E70757420747970653D22737562E6
:100320006D697422207374796C653D226865696714
:1003300068743A203530707822206E616D653D22F8
:10034000746F67676C65222076616C75653D224C21
:10035000454437222F3E266E627370266E6273709C
:100360003C2F6669656C647365743E3C2F666F72E2
:100370006D3E3C2F74643E3C74643E266E62737026
:100380003B3C2F74643E3C2F74723E3C2F74616280
:100390006C653E3C2F74643E3C74642077696474E1
:1003A000683D323025253E3C2F74643E3C2F7472EC
:1003B0003E3C2F7461626C653E3C2F626F64793EF7
:1003C0003C2F68746D6C3E003C74723E3C74643E1D
:1003D0003C666F726D206D6574686F643D22676561
:1003E00074223E3C696E70757420747970653D228C
:1003F0007375626D697422207374796C653D22682F
:1004000065696768743A2035307078222076616CAF
:1004100075653D2252656672657368222F3E3C2FDA
:10042000666F726D3E3C2F74643E3C2F74723E3C8E
:100430002F7461626C653E3C62723E3C666F726D09
:100440002069643D22666F726D226E616D653D228A
:10045000666F726D22206D6574686F643D226765FA
:10046000742220616374696F6E3D22696E646578E1
:100470002E68746D6C223E3C6669656C64736574AD
:10048000207374796C653D2277696474683A20330F
:1004900030303B223E3C6C6567656E643E4C4544A3
:1004A00020636F6E74726F6C3C2F6C6567656E6451
:1004B0003E3C696E70757420747970653D22737569
:1004C000626D697422207374796C653D2268656978
:1004D0006768743A203530707822206E616D653D12
:1004E00022746F67676C65222076616C75653D22AA
:1004F0004C454430222F3E266E627370266E627326
:10050000703C696E70757420747970653D227375E6
:10051000626D697422207374796C653D2268656927
:100520006768743A203530707822206E616D653DC1
:1005300022746F67676C65222076616C75653D2259
:100540004C454431222F3E266E627370266E6273D4
:10055000703C696E70757420747970653D22737596
:10056000626D697422207374796C653D22686569D7
:100570006768743A203530707822206E616D653D71
:1005800022746F67676C65222076616C75653D2209
:100590004C454432222F3E266E627370266E627383
:1005A000703C696E70757420747970653D22737546
:1005B000626D697422207374796C653D2268656987
:1005C0006768743A203530707822206E616D653D21
:1005D00022746F67676C65222076616C75653D22B9
:1005E0004C454433222F3E266E627370266E627332
:1005F000703C703E003C2F74643E3C74643E3C6230
:100600003E3C2F623E3C2F74643E3C2F74723E0091
:100610003C74723E3C74643E54656D7065726174E6
:100620007572653A20003C2F74643E3C74643E3C15
:10063000623E3C2F623E3C2F74643E3C2F74723EFF
:10064000003C74723E3C74643E4D414320416464FE
:10065000726573733A20003C2F74643E3C74643EB0
:100660003C623E3C2F623E3C2F74643E3C2F7472D1
:100670003E003C74723E3C74643E495020416464C8
:10068000726573733A2000485454502F312E302035
:10069000323030204F4B0A5365727665723A2077BC
:1006A0006C705F68747470640A436F6E74656E7406
:1006B0002D747970653A20746578742F68746D6C48
:1006C0000A0A3C21444F43545950452048544D4C4C
:1006D000205055424C494320222D2F2F5733432F72
:1006E0002F4454442048544D4C20342E3031204661
:1006F00072616D657365742F2F454E2220226874D8
:1007000074703A2F2F7777772E77332E6F72672F8B
:1007100054522F68746D6C342F6672616D65736509
:10072000742E647464223E3C68746D6C3E3C686553
:1007300061643E3C7469746C653E6F574C2070690F
:10074000636F204854545020576562207365727659
:1007500065723C2F7469746C653E3C2F68656164FA
:100760003E3C626F6479207374796C653D666F6E90
:10077000742D66616D696C793A617269616C3E3C99
:100780007461626C653E3C74723E3C7464207769AF
:100790006474683D3130303E3C2F74643E3C746478
:1007A0003E3C7461626C653E3C74722076616C699B
:1007B000676E3D22746F70223E3C746420776974CA
:1007C000683E3C696D67207372633D226C6F676F92
:1007D0002E6769662220626F726465723D22302244
:1007E00020616C743D226C6F676F227469746C6554
:1007F0003D226C6F676F223E3C2F74643E3C2F7429
:10080000723E3C74723E3C74642077696474683D47
:1008100022353030223E3C68323E576562205365B7
:10082000727665722072756E6E696E67206F6E20CB
:100830006F574C207069636F3C2F68323E3C703EAE
:100840005468652077656220706167652069732050
:1008500073657276656420627920776C705F687466
:10086000747064207573696E6720746865205350D6
:100870004238303020574C414E206D6F64756C65A6
:1008800020616E6420746865206F574C2D70696319
:100890006F26636F70793B20536F66747761726562
:1008A000204150493B206120756E69717565205764
:1008B000692D466920736F6C7574696F6E2066725E
:1008C0006F6D203C623E48264420576972656C6516
:1008D00073732041423C2F623E2E3C2F703E3C6899
:1008E000723E3C7461626C653E004749463839612E
:1008F00045017B00A10000FFFFFF0066990000009A
:10090000FFFFFF21FE114372656174656420776902
:1009100074682047494D50002C0000000045017BC1
:10092000000002FE848FA9CBED0FA39CB4DA8BB339
:10093000DEBCFB0F86E24896E689A6EACAB6EE0B55
:10094000C7F24CD7F68DE7FACEF7FE0F0C0A87C434
:10095000A2F1884C2A97CCA6F3098D4AA7D4AAF510
:100960008A6505B6DCAEF70B0E8BC76471F60C2DED
:10097000ABD7EC36190D3FBAE7F4FA3B8EFFD9F747
:100980007C7BFE9FD32738C80668384398A8187622
:10099000D8D8B2081919E048792279A958A929822A
:1009A000D929B809DAE139CA176A8A419A4A77CA55
:1009B0003AA1FAEAD62AEB005BAB368BAB60BB6B95
:1009C00096EB0BC01BECF5EB2B6CBC458C7B6C9C4D
:1009D0003CBB2CDC2CFB1C1CDD3ACD5BCD7ABD9BDB
:1009E0007DBA6DDB6DFA5D1B1E3A0E5B0E7AFE9AC8
:1009F000BEB9AEDAAEF99E1A5F394F5A4F793F9AB7
:100A0000EFB8EFD9AFD1BF4E010F0DC454D0D0C154
:100A10004B09012D94D4F0CFC34811F34C845411E9
:100A2000CF1DFE5D601A8CF158A6421B04024A9A43
:100A300014B0E0E4C9942A511E68290366B88D09F0
:100A40001831B0F980A6AB5B2465F6F4F9122800E2
:100A5000A12D8836D3790027C761123E5EE0195474
:100A6000A5829625A70A35BA022B31A40694D6642E
:100A7000DAB4D7539D5413503569F6AAD4185A7F67
:100A80007105D6F126D8B07151398DBAF26759BDCA
:100A900068F9BA84D1B6D8DDAF5F4072913B69691D
:100AA000E10C64D59E4DBB7647E05C6FBD22987B20
:100AB000199962CC490FD3128BB7AF81B355FDFAA8
:100AC00098AC6C70E6C50B58AFDECCB96B6CD996A0
:100AD000F70E255DFA76E4D07F47FBCCCB12788306
:100AE000C9A879E77EF0B847E5BAB05B2726CC7C89
:100AF0007517C4D17503C79DDB366FC82B8962EFAC
:100B0000CDFD7878ED56B10FFFCEE3ADC8D9CE411B
:100B10004BF7DCDEB5EFC8E8E70BB72FBE2CD0EF04
:100B2000F7FEF183F78F5B70FC95376020AAD9C57B
:100B3000DE7BD5D1361D75B1FD661E8004E65720DB
:100B400080018E2760851692365E8438A847C18260
:100B5000D0B9D7197B245A87964C2AEEB69D5FDA16
:100B6000F1C7228AFFC1789F63C2D9289A0D20EE6F
:100B7000045F4E21C5D7E3880D7628A37F32FE5748
:100B8000A48B10C6481E8EE21D69DA04C5DDB023B1
:100B90005DCF41009F8822C2B5A07E6BC1449E916B
:100BA0004A228995931866D85B98E7C5E843951162
:100BB0000489E0950ACA39A7661DDAA6618BC621A9
:100BC00079248C51EE59619E63F6F7E1810C0EB9E0
:100BD0001407B36D79629F377A78E69E0CD0B81F00
:100BE0008B94EE46239A1CEAB09C7C9921C6239DE7
:100BF00087DA091B9C1BE658DF84E0A9792AA44EFA
:100C0000663A289BB016DAA8659D01F926A2733AC8
:100C1000385BAA8EE6F8A784935E8AAAA5C43EF93B
:100C2000FE2BA1C9024B43A7268AEAA990BC1A262B
:100C300022A4AD0E5BA356AC3A60A6079B22F76DCB
:100C40000DCEEAFA2990A46E469D8FB69EAA2A9BE5
:100C5000491AB7A6B2DC1AEB6E0653BEABA3A15C71
:100C60003E6B188F1BE8FB6BBBCCEA29ACA6AB76BE
:100C70002BA98B146CABAA81B5322A2A63115BB9FC
:100C8000E58583C64B61BDCB7AC724B109EB991CBE
:100C9000C1E2EABB2E971E984A71C521DFC927BE63
:100CA00050622C28C794B21CAEC7B4AE5B32B916E2
:100CB000E89CAB7AE18E093391F3FAD9B0C02BB737
:100CC000FAAAC554920C31CAEDBD37D68FD8BAFBFB
:100CD00073B02F83AB74A4460F0C28D5828EFC70A2
:100CE000B4A34EBC6F8309960AF0D59A0E0D2CC39F
:100CF00045B38DACD0111C0D73CBF95E9448467191
:100D0000E09D89DE68F09DB7DF67004E88E08313C1
:100D1000FE89E158209EB8E25630DE87E35740ADA9
:100D20005E8AE45550BE87E597635E87E65470DEC1
:100D3000B9E75280BE8AE851903E87E9A7A33E9268
:100D4000EA4FB0DEBAEB4DC05E88ECB3D30E95ED42
:100D50004AE09EBBEE48F02EB5EFBF039FB6F040D1
:100D6000105FBCF16D225FB2F27A30BFA5F3CB43C6
:100D70007FB6F43B505FBDF59C62EFB4F6CA714F8D
:100D8000B6F7D7832F3E11E4976F3EF6E8A74FFDE5
:100D9000FAEC23EF7E11CCC72F3FF1F41B01FCFDD1
:100DA000C3B3AE7F12A4F77F3BC601F0730719A04F
:100DB000010F88C0042A70810C6CA0031F08C108B1
:100DC0004A708214ACA0052F8841CD1500003B4825
:100DD0005454502F312E3020323030204F4B0A5394
:100DE00065727665723A20776C705F6874747064AF
:100DF0000A436F6E74656E742D747970653A20695C
:100E00006D6167652F6769660A0A00485454502F60
:100E1000312E30203430342046696C65206E6F747A
:100E200020666F756E640A5365727665723A207734
:100E30006C705F68747470640A436F6E74656E746E
:100E40002D747970653A20746578742F68746D6CB0
:100E50000A0A3C68746D6C3E3C686561643E3C7493
:100E600069746C653E6F574C207069636F204854FD
:100E7000545020576562207365727665723C2F74FA
:100E800069746C653E3C2F686561643E3C626F64CA
:100E9000793E3C68323E343034202D205061676505
:100EA000206E6F7420666F756E643C2F68323E3C16
:100EB000703E536F7272792C207468652070616780
:100EC0006520796F75206172652072657175657333
:100ED00074696E6720776173206E6F7420666F751A
:100EE0006E64206F6E207468697320736572766516
:100EF000722E3C2F703E3C2F626F64793E3C2F680F
:100F0000746D6C3E006364696E6F70737578585BC6
:100F1000000011241FBECFEFDFE3DEBFCDBF00E036
:100F20000CBF18BE19BE1ABE1BBE1BE2A0E0B0E289
:100F3000E6E4F8E800E00BBF02C007900D92AE3D7A
:100F4000B107D9F71BBE1CE2AEEDBBE201C01D929A
:100F5000A532B107E1F70E9409320C9421440C94A8
:100F600000009BB78BBFFB018091CA014093CA016F
:100F70007DE970933400E8958093CA019BBF089582
:100F80002091CF0127FDFCCF9BB78BBFFB01809148
:100F9000CA0123E22093CA010A01E8951124809333
:100FA000CA019BBF0895FC019FB7F894E059FF4F19
:100FB00060958081862380839FBF0895FC019FB741
:100FC000F894E059FF4F8081862B80839FBF08955E
:100FD000E0E7F0E08FEF8193E737F105E1F79FB7A6
:100FE000F894809150008260809350009FBF809160
:100FF000510081FFFCCF80E490E061E00E94FA3173
:101000009FB7F894809150008E7F809350009FBFCF
:101010000895282FAB0186958695869590E0C09619
:10102000277061E070E002C0660F771F2A95E2F733
:1010300025E0880F991F2A95E1F70E9485080895F9
:1010400080E260E073E00E94090881E260E073E002
:101050000E94090882E260E073E00E94090883E2CE
:1010600060E073E00E94090884E260E073E00E949F
:10107000090885E260E073E00E94090886E260E00A
:1010800073E00E94090887E260E073E00E940908AB
:1010900088E268E170E00E94090889E268E170E096
:1010A0000E9409088AE268E170E00E9409088BE268
:1010B00068E170E00E9409088CE268E170E00E943B
:1010C00009088DE268E170E00E9409088EE268E19B
:1010D00070E00E9409088FE268E170E00E94090850
:1010E00083E160E073E00E94090882E160E070E063
:1010F0000E9409088BE160E073E00E9409088AE120
:1011000060E070E00E9409080895CF93DF93DC014E
:10111000FC0120E030E0C62FD0E0CE01022E02C05C
:10112000959587950A94E2F780FD408B2F5F3F4F9E
:1011300031962830310589F750FF0CC051FF04C0AB
:1011400015966C93159703C016966C931697119687
:101150006C9302C012966C93DF91CF9108959B011E
:10116000AC01109200048091010480FDFCCFE0E00E
:10117000F4E020873187CA01AA27BB278093042C7B
:101180009093052C87E08093000408959FB7F8940E
:101190002091042C3091052C609108047091090471
:1011A0006115710531F48091030480FF02C02F5F47
:1011B0003F4F9FBF40E050E0A90133272227CB01DA
:1011C000A0E0B0E0282B392B4A2B5B2BB901CA01D8
:1011D00008959B01AC0181E0E0E0F4E0828380911E
:1011E000010480FDFCCFE0E0F4E024873587209304
:1011F000082C3093092CCA01AA27BB278093062C00
:101200009093072C8091010480FDFCCF85E0E0E005
:10121000F4E082830895E0E0F4E08281869586958B
:1012200080958170089580930A2C90930B2C0895DB
:101230001F920F920FB60F9208B60F9218BE11248C
:101240008F939F938091042C9091052C019680930D
:10125000042C9093052C9F918F910F9008BE0F90B6
:101260000FBE0F901F9018951F920F920FB60F92FE
:1012700008B60F9218BE09B60F9219BE0BB60F92A0
:101280001BBE1124EF92FF920F931F932F933F9356
:101290004F935F936F937F938F939F93AF93BF937E
:1012A000EF93FF932091042C3091052C6091062C34
:1012B0007091072C26173707C0F181E0E0E0F4E0D9
:1012C0008283E0910A2CF0910B2C309771F1809180
:1012D00008049091090440E050E08901FF24EE24C5
:1012E000A0E0B0E0E82AF92A0A2B1B2BCB01A0E0F2
:1012F000B0E0AC01332722278091082C9091092C73
:10130000A0E0B0E0282B392B4A2B5B2B2E153F0594
:101310004007510738F079018A010894E11CF11C5B
:10132000011D111DC801B7011995FF91EF91BF91E2
:10133000AF919F918F917F916F915F914F913F916D
:101340002F911F910F91FF90EF900F900BBE0F9078
:1013500009BE0F9008BE0F900FBE0F901F901895FA
:1013600080E090E064E00E94D30721E0E0E4F0E058
:101370002383E0E0F4E08FEF9FEF8287938710866E
:101380001186228387E080830895E091E02BF0911D
:10139000E12B87839087618772870895E091E02B26
:1013A000F091E12B8387948765877687089586EF90
:1013B0009FEF0895AF92BF92CF92DF92EF92FF928C
:1013C0000F931F93DF93CF930F920F92CDB7DEB79A
:1013D0006C01162F072F7A0159011F5F19831150D5
:1013E000E091E02BF091E12B228133818481958182
:1013F000BE016F5F7F4F41E050E0F9011995E09128
:10140000E02BF091E12B2081318184819581BE0117
:101410006E5F7F4F41E050E0F90119959A81898113
:10142000981719F020EF3FEF23C0E091E02BF091E7
:10143000E12B2281338184819581B601412F502F88
:10144000F9011995E091E02BF091E12B2081318198
:1014500084819581B701A501F9011995F701808172
:1014600091810E94F211F7018083918320E030E0A6
:10147000C9010F900F90CF91DF911F910F91FF90B5
:10148000EF90DF90CF90BF90AF9008952F923F9252
:101490004F925F926F927F928F929F92AF92BF9284
:1014A000CF92DF92EF92FF920F931F93DF93CF9330
:1014B000CDB7DEB76997CDBFDEBF5C014B013A0106
:1014C00029011701760188E08983CE01019661E048
:1014D00070E0AE014E5F5F4F28E130E00E94DA0914
:1014E0009C0197FD52C0A114B10449F08E819F81E7
:1014F000A885B985F50180839183A283B383811484
:10150000910449F08A859B85AC85BD85F401808373
:101510009183A283B3836114710449F08E859F8502
:10152000A889B989F30180839183A283B38341148D
:10153000510449F08A899B89AC89BD89F201808375
:101540009183A283B3830115110539F08D81992709
:1015500087FD9095F80180839183E114F10439F0BF
:101560008C81992787FD9095F701808391832114C1
:10157000310449F08E899F89A88DB98DF10180834E
:101580009183A283B3832A813B81C9016996CDBF30
:10159000DEBFCF91DF911F910F91FF90EF90DF9011
:1015A000CF90BF90AF909F908F907F906F905F9003
:1015B0004F903F902F900895CF92DF92EF92FF923D
:1015C0000F931F938C0180E090E060E070E040E0BA
:1015D00050E020E030E0EE24FF24CC24DD240E9403
:1015E000460A1F910F91FF90EF90DF90CF900895E2
:1015F000CF92DF92EF92FF920F931F9300E010E0E3
:10160000EE24FF24CC24DD240E94460A1F910F9172
:10161000FF90EF90DF90CF9008950F93DF93CF93DB
:10162000CDB7DEB76697CDBFDEBFFC0187E08B8309
:10163000309749F080819181A281B3818F8398870F
:10164000A987BA8704C01F82188619861A86611571
:10165000710551F0FB0180819181A281B3818B875B
:101660009C87AD87BE8704C01B861C861D861E8690
:101670004115510551F0FA0180819181A281B38118
:101680008F87988BA98BBA8B04C01F86188A198AFA
:101690001A8A2115310551F0F90180819181A281C9
:1016A000B3818B8B9C8BAD8BBE8B04C01B8A1C8A39
:1016B0001D8A1E8A0E83CE01039664E170E0AE019E
:1016C0004F5F5F4F22E030E00E94DA099C0197FDF6
:1016D00002C029813A81C9016696CDBFDEBFCF9194
:1016E000DF910F9108950F931F938C0180E090E09C
:1016F00060E070E040E050E020E030E00E940D0B40
:101700001F910F9108950F931F9300E010E00E9426
:101710000D0B1F910F910895DF93CF9300D0CDB79C
:10172000DEB783E08983CE01019661E070E0AE010F
:101730004E5F5F4F22E030E00E94DA099C0197FD86
:1017400002C02A813B81C9012396CDBFDEBFCF9164
:10175000DF9108950F931F93DF93CF93CDB7DEB73B
:101760002C97CDBFDEBF8B0124E129830E94EE11AF
:101770008B839C83CE01019664E070E0AE014B5FE9
:101780005F4F28E030E00E94DA099C0197FD0DC010
:101790002D813E8137FD09C089859A85AB85BC8541
:1017A000F80180839183A283B383C9012C96CDBFB6
:1017B000DEBFCF91DF911F910F910895EF92FF92BD
:1017C0000F931F93DF93CF93CDB7DEB72897CDBF8D
:1017D000DEBF7B018A0120E12B830E94EE118D8305
:1017E0009E83C8010E94EE118F839887CE010396D5
:1017F00066E070E0AE014F5F5F4F22E030E00E9494
:10180000DA09AC0197FD16C049815A8157FD12C013
:10181000041715071CF440EF5FEF0CC0E091E02BBC
:10182000F091E12B2281338184819581B701F90107
:101830001995AC01CA012896CDBFDEBFCF91DF91CB
:101840001F910F91FF90EF900895EF92FF920F93E9
:101850001F93DF93CF93CDB7DEB72897CDBFDEBF01
:101860007B018A012FE02B830E94EE118D839E83E2
:10187000C8010E94EE118F839887CE01039666E01F
:1018800070E0AE014F5F5F4F22E030E00E94DA0966
:10189000AC0197FD16C049815A8157FD12C004174B
:1018A00015071CF440EF5FEF0CC0E091E02BF091C6
:1018B000E12B2081318184819581B701F90119954E
:1018C000AC01CA012896CDBFDEBFCF91DF911F9139
:1018D0000F91FF90EF9008956F927F928F929F9259
:1018E000AF92BF92CF92DF92EF92FF920F931F932E
:1018F000DF93CF93CDB7DEB72C97CDBFDEBFFC0112
:101900006B015A01490138010091E22B1091E32B40
:101910000BC0D8018D919C9111978E179F0751F0A4
:1019200013960D911C9114970115110591F72EEF47
:101930003FEF34C08DE08B83CF010E94EE118D8389
:101940009E83F60180819181A281B3818F839887E4
:10195000A987BA87C5010E94EE118B879C87CE01AB
:1019600003966AE070E0AE014F5F5F4F22E030E027
:101970000E94DA099C0197FD11C029813A8137FD47
:101980000DC0D80117968D929C92189719966D925A
:101990007C921A971B96ED92FC921C97C9012C968B
:1019A000CDBFDEBFCF91DF911F910F91FF90EF90E0
:1019B000DF90CF90BF90AF909F908F907F906F906F
:1019C00008951F93DF93CF9300D000D0CDB7DEB73B
:1019D000DC01162FE091E22BF091E32B08C080810F
:1019E00091818A179B0741F00380F481E02D3097A5
:1019F000B1F72EEF3FEF1CC0458356832387348712
:101A00008CE08B83CD010E94EE118D839E831C831D
:101A1000CE01039664E070E0AE014F5F5F4F22E0BD
:101A200030E00E94DA099C0197FD02C029813A81C9
:101A3000C9012696CDBFDEBFCF91DF911F910895DA
:101A4000EF92FF920F931F93DF93CF93CDB7DEB743
:101A50002C97CDBFDEBF8B017A012BE02B830E9438
:101A6000EE118D839E83F80180819181A281B381E3
:101A70008F839887A987BA87C7010E94EE118B8749
:101A80009C87CE0103966AE070E0AE014F5F5F4F26
:101A900022E030E00E94DA099C0197FD02C0298112
:101AA0003A81C9012C96CDBFDEBFCF91DF911F9146
:101AB0000F91FF90EF900895AF92BF92CF92DF9277
:101AC000EF92FF920F931F93DF93CF93CDB7DEB7C3
:101AD0006597CDBFDEBF8091E02B9091E12B892BE4
:101AE00009F4A0C184E08983CE01019661E070E031
:101AF000AE014C5F5F4F22E030E00E94DA0997FDB3
:101B000019C08C819D81009799F4E091E02BF091B0
:101B1000E12B278130852115310501F1868180FD7A
:101B20001DC0816086838185928561E070E014C06C
:101B300097FF14C0E091E02BF091E12B27813085D5
:101B40002115310559F0868180FF08C08E7F86837C
:101B50008185928560E070E0F9011995A6E0AA2ED2
:101B6000B12CAC0EBD1EC50160E070E040E050E05D
:101B700020E030E000E010E0FAE0EF2EF12CEC0E77
:101B8000FD1EE2E0CE2ED12CCC0EDD1E0E94460AB8
:101B90000097A1F4E091E02BF091E12B23853485AF
:101BA0002115310521F1868181FD21C08260868366
:101BB00085859685B501F901199519C097FF15C05E
:101BC000E091E02BF091E12B23853485211531053F
:101BD000A9F1868181FF32C08D7F868385859685B8
:101BE00060E070E0F901199529C0892B39F5E09181
:101BF000E02BF091E12B2785308921153105F1F09B
:101C00008A819B81009731F481899289BE01665F48
:101C10007F4F07C08F5F9F4F31F48189928960E0C9
:101C200070E0F90119958A819B818E5F9F4F31F099
:101C3000E091E02BF091E12B1786108AE091E02BE8
:101C4000F091E12B8681846086830091E22B1091D4
:101C5000E32B22E1B22E9EE0C92ED12CCC0EDD1E4C
:101C600082E1E82EF12CEC0EFD1E98C0F801808177
:101C70009181BE860E94EE11888B998BC60164E02B
:101C800070E0A70124E030E00E94DA0997FD81C0EE
:101C90009D894A895B8957FD7CC09130D1F4D80178
:101CA00012968C91129780FD44C01796ED91FC918D
:101CB00018973097F1F1816012968C9312976D917D
:101CC0007C9111971B968D919C911C9741E050E05F
:101CD00041C09430E1F4D8011796ED91FC9118972A
:101CE000309739F112968C9112978E7F12968C93C1
:101CF00012976D917C9111971B968D919C911C97D9
:101D000040E050E01995F8011782108642C09330E8
:101D100081F4D8011596ED91FC911697309749F012
:101D20006D917C9111971B968D919C911C971995A3
:101D300030C04115510581F0D8011996ED91FC9103
:101D40001A97309749F06D917C9111971B968D9160
:101D50009C911C9719951DC09923D9F4F801828193
:101D600080FF17C00184F285E02D309791F08E7FBF
:101D7000D80112968C9312976D917C9111971B96B6
:101D80008D919C911C9740E050E01995F8011186C7
:101D90001286D80113960D911C9114970115110507
:101DA00009F064CFE091E02BF091E12B86818B7FED
:101DB0008683A091E22BB091E32BEE24FF2430C068
:101DC00012968C91129781FF23C0E114F10459F40B
:101DD000E091E22BF091E32B838194818093E22BBD
:101DE0009093E32B07C013968D919C911497F70164
:101DF0008383948313961C91139714960C911497D4
:101E0000CD010E949E3A212F302FC901DC0108C06C
:101E10007D0113968C91139714969C919C01D90186
:101E2000109771F66596CDBFDEBFCF91DF911F9100
:101E30000F91FF90EF90DF90CF90BF90AF900895FB
:101E40000F931F93DF93CF9300D000D0CDB7DEB7B1
:101E50008C018EE08B83C8010E94EE118D839E83DE
:101E6000CE01039664E070E0AE014F5F5F4F22E069
:101E700030E00E94DA099C0197FD42C029813A8135
:101E800037FD3EC06091E22B7091E32BDB0140E017
:101E900050E032C08D919C9111978017910721F5E8
:101EA000E091E02BF091E12B868182FF07C0129632
:101EB0008C911297826012968C9320C04115510527
:101EC00041F4FB01838194818093E22B9093E32B77
:101ED00007C013968D919C911497FA018383948384
:101EE000CD010E949E3A0AC0AD0113968C911397C2
:101EF00014969C919C01D901109761F620E030E086
:101F0000C9012696CDBFDEBFCF91DF911F910F9102
:101F10000895EF92FF920F931F93DF93CF93CDB766
:101F2000DEB7C358D040CDBFDEBF9C018B017A0124
:101F30000097C1F1FC0101900020E9F73197E81BFF
:101F4000F90BE038F10570F5E091E02BF091E12B11
:101F500087859089892B19F022EF3FEF25C089E012
:101F60008B83CE010496B9010E94723DCE01039687
:101F700061E870E0AE014F5F5F4F22E030E00E9409
:101F8000DA099C0197FD10C029813A81211531059C
:101F900059F4E091E02BF091E12B0787108BE18A57
:101FA000F28A02C02EEF3FEFC901CD57DF4FCDBF00
:101FB000DEBFCF91DF911F910F91FF90EF900895B9
:101FC0008F929F92AF92BF92CF92DF92EF92FF9249
:101FD0000F931F93DF93CF9300D000D0CDB7DEB720
:101FE0007C014B016A01590181E090E06DE070E0F5
:101FF0000E94D5398C01009729F4BDEFEB2EBFEF7D
:10200000FB2E48C083E18B83C7010E94EE118D83B4
:102010009E83CE01039664E070E0AE014F5F5F4F98
:1020200022E030E00E94DA097C0197FF04C0C80179
:102030000E949E3A2FC089819A8197FF06C0C801ED
:102040000E949E3AE980FA8025C0F801808391833E
:1020500013821482C186D28687829086A386B48634
:10206000828181608283E091E22BF091E32B3097B3
:1020700029F40093E22B1093E32B09C0CF010380D6
:10208000F481E02D3097D1F7FC0103831483F8012C
:10209000E080F180C7012696CDBFDEBFCF91DF91F2
:1020A0001F910F91FF90EF90DF90CF90BF90AF9076
:1020B0009F908F900895EF92FF920F931F93DF935D
:1020C000CF93CDB7DEB72597CDBFDEBF182F672BD7
:1020D00019F006EF1FEF48C081E090E06DE070E07E
:1020E0000E94D5397C01009719F40DEF1FEF3CC019
:1020F0008AE08B831C831D82CE01039663E070E02F
:10210000AE014F5F5F4F22E030E00E94DA098C01A0
:1021100097FF04C0C7010E949E3A26C089819A8118
:1021200097FF06C0C7010E949E3A09811A811CC010
:10213000F7018083918313821482E091E22BF09166
:10214000E32B309729F4E092E22BF092E32B09C0C5
:10215000CF010380F481E02D3097D1F7FC01E382B9
:10216000F482F70100811181C8012596CDBFDEBF41
:10217000CF91DF911F910F91FF90EF9008950F93F2
:102180001F93DF93CF93CDB7DEB7E397CDBFDEBF0D
:102190008C0185E08983CE01019661E070E0AE019B
:1021A0004E5F5F4F22E330E00E94DA099C0197FD09
:1021B00016C00115110589F0D8019196FE013C96D3
:1021C00086E001900D928150E1F7D801FE017296F0
:1021D00081E201900D928150E1F72A813B81C90192
:1021E000E396CDBFDEBFCF91DF911F910F91089590
:1021F0000F931F93DF93CF93CDB7DEB7E397CDBF98
:10220000DEBF8C0185E08983CE01019661E070E03C
:10221000AE014E5F5F4F22E330E00E94DA099C017D
:1022200097FD0DC00115110541F0D801FE0136964C
:1022300086E001900D928150E1F720E030E0C90185
:10224000E396CDBFDEBFCF91DF911F910F9108952F
:102250001F93DF93CF93CDB7DEB7C856D040CDBF25
:10226000DEBF9C01142F86E6FE013396DF011D922E
:102270008A95E9F782E08B832115310541F0DE0173
:102280001796F90181E201900D928150E1F76115F5
:10229000710531F0CE0188964FE350E00E94873DF2
:1022A000FE01E859FF4F1083CE01039666E670E009
:1022B000AE014F5F5F4F22E030E00E94DA099C01DF
:1022C00097FD02C029813A81C901C859DF4FCDBFAE
:1022D000DEBFCF91DF911F9108959F92AF92BF9281
:1022E000CF92DF92EF92FF920F931F93DF93CF93E2
:1022F000CDB7DEB72B97CDBFDEBF5B016C01942E4F
:10230000D801C70147E749836CE07CE26093E02B8A
:102310007093E12B43E1FB0111924A95E9F7209379
:102320000C2C30930D2C00930E2C10930F2CE0925C
:10233000102CF092112C8E010F5F1F4FB80141E05D
:1023400050E0FD011995E091E02BF091E12B208107
:10235000318184819581B80141E050E0F9011995FE
:10236000F02E012F0EC0E091E02BF091E12B2081A7
:102370003181848195816F2D702F41E050E0F9010A
:10238000199589818E3279F31C82C601B5010E94AC
:10239000F611688779878A879B879F82CE0104968A
:1023A00068E070E0AE014E5F5F4F22E030E00E94D7
:1023B000DA099C0197FD02C02A813B81C9012B9655
:1023C000CDBFDEBFCF91DF911F910F91FF90EF90B6
:1023D000DF90CF90BF90AF909F900895282F892FC6
:1023E000922F0895282F892F922F0895EF92FF9210
:1023F0000F931F93E92EFF2400271127562F442700
:1024000033272227E22AF32A042B152B2227362FE3
:10241000472F582F207030705070E22AF32A042B77
:10242000152B672F782F892F9927607080709070F7
:10243000E62AF72A082B192BB701C8011F910F9123
:10244000FF90EF900895EF92FF920F931F93E92E64
:10245000FF2400271127562F442733272227E22A5B
:10246000F32A042B152B2227362F472F582F2070A5
:1024700030705070E22AF32A042B152B672F782F27
:10248000892F9927607080709070E62AF72A082BB0
:10249000192BB701C8011F910F91FF90EF9008957C
:1024A0002F923F924F925F926F927F928F929F9264
:1024B000AF92BF92CF92DF92EF92FF920F931F9352
:1024C000DF93CF93CDB7DEB76497CDBFDEBFFC01FE
:1024D000698B7A8B8081C82EDD24C7FCD0944E0195
:1024E0000894811C911C9E01235F3F4F2B8B3C8BDA
:1024F0008C2D80538A3008F067C130E3C316D104B5
:1025000021F09AE0692E712C1BC031968081C82E73
:10251000DD24C7FCD09448E7C416D10441F058E547
:10252000C516D10421F088E0682E712C09C03196BF
:102530008081C82EDD24C7FCD09400E1602E712C70
:102540005F010894A11CB11CEE24FF248701130134
:10255000442437FC4094542CD50111979C2D8C2D8C
:1025600080538A30A0F4C801B701A20191010E94F2
:102570006139E0EDFFEFCE0EDF1E76010027F7FC9C
:102580000095102FE60EF71E081F191F2BC0F0E153
:102590006F16710489F52C2D2156263048F08C2DAC
:1025A0008154863048F52A3118F021E430E002C029
:1025B00021E630E0D801C70114E0880F991FAA1F57
:1025C000BB1F1A95D1F74AE050E0C40ED51EC21ABF
:1025D000D30A76010027F7FC0095102FE82AF92A84
:1025E0000A2B1B2BF5018081C82EDD24C7FCD0945B
:1025F0000894A11CB11CB0CFFEE2CF16D104C1F4E7
:102600002B893C898216930609F4DEC0F401E0822E
:10261000F1820283138324E030E0820E931EFD01D9
:10262000319611968C91C82EDD24C7FCD09460CFD2
:10263000C114D104F1F0903208F4C6C0C7FCC4C084
:1026400030E2C316D104A9F04CE0C416D10489F0DD
:102650005AE0C516D10469F08DE0C816D10449F0DE
:1026600099E0C916D10429F0EBE0CE16D10409F0A7
:10267000ABC0CE0101969401281B390BC901959579
:1026800087959595879501968230910571F08330F5
:10269000910524F4892B09F497C067C08330910514
:1026A000B9F0049709F061C035C030E0E31630E0BE
:1026B000F30630E0030731E0130708F085C0898195
:1026C0009A81AB81BC81B82FAA279927882749C056
:1026D00040E0E41640E0F40641E0040740E014075F
:1026E00008F072C02D813E814F815885A9013327A2
:1026F000222789819A81AB81BC81B82FAA2799278B
:102700008827282B392B4A2B5B2BE22AF32A042B10
:10271000152B2BC05FEFE516F1040105110511F033
:1027200008F052C08D819E81AF81B885DC01992768
:10273000882729813A814B815C81522F4427332796
:102740002227822B932BA42BB52B29853A854B85E9
:102750005C85542F432F322F2227822B932BA42BBF
:10276000B52BE82AF92A0A2B1B2B89899A89892BF0
:1027700041F1212F332744275527BE2DAA2799271A
:102780008827282B392B4A2B5B2BB02FAF2D9E2D62
:10279000882780709070B070282B392B4A2B5B2BC8
:1027A000BB27A12F902F8F2D8070A070B070282B89
:1027B000392B4A2B5B2BE989FA89208331834283A9
:1027C000538321E030E002C020E030E0C90164968C
:1027D000CDBFDEBFCF91DF911F910F91FF90EF90A2
:1027E000DF90CF90BF90AF909F908F907F906F9031
:1027F0005F904F903F902F900895AF92BF92CF92ED
:10280000DF92EF92FF920F931F93DF93CF93CDB799
:10281000DEB72797CDBFDEBFFC0180819181A28109
:10282000B3818C839D83AE83BF8334E0E32EF12C90
:10283000EC0EFD1E04EE1BE26E010894C11CD11CBF
:102840005EE227E0A22EB12CAC0EBD1ED7014C914A
:1028500030E0842F6AE00E948039292F842F0E9463
:102860008039482FF601E30FF11D205D20833F5F83
:10287000882379F7932FF7011082D80106C03150D1
:10288000F601E30FF11D80818D933323C1F7F80129
:10289000E90FF11DDF015D938D01EA14FB0421F0C6
:1028A0000894E11CF11CD2CF108284EE9BE22796A3
:1028B000CDBFDEBFCF91DF911F910F91FF90EF90C1
:1028C000DF90CF90BF90AF900895CF93DF93EC014E
:1028D000DB0116964D935C931797EA81FB81309745
:1028E00019F46A837B8309C0CF010084F185E02D50
:1028F0003097D1F7FC01A087B18718961D921C92E2
:102900001997DF91CF910895FB0146835783DC012E
:102910009C966D937C939D970895FC018081918195
:102920000895CF92DF92EF92FF920F931F93CF9370
:10293000DF938C016B017A01C0E0D0E012C0F60198
:10294000EC0FFD1F6081772767FD7095D801169603
:10295000ED91FC91179718968D919C911997199567
:102960002196CE15DF055CF3DF91CF911F910F917A
:10297000FF90EF90DF90CF900895AF92BF92CF92EB
:10298000DF92EF92FF920F931F93CF93DF93FC019F
:102990008B01DB018C91882319F4C0E0D0E02DC0BD
:1029A000C281D381EE24FF24AA24BB2421C0C88085
:1029B000D980C601B8010E94693D0097F1F0D801A5
:1029C0000D900020E9F71197A01BB10BC601B801CB
:1029D000AD010E94793D009741F4EF2829F07E0176
:1029E00081E0A82EB12C01C07E010884D985C02DBC
:1029F0002097E9F6AB2809F4E701CE01DF91CF91EA
:102A00001F910F91FF90EF90DF90CF90BF90AF900C
:102A10000895CF93DF93EC01009749F08A859B8559
:102A2000009711F00E949E3ACE010E949E3ADF91DB
:102A3000CF9108958F929F92AF92BF92CF92DF92E3
:102A4000EF92FF920F931F93CF93DF934C01162FBA
:102A5000072F81E090E061E070E00E94D539EC0141
:102A6000009709F44AC0812F902F9C018901CC2442
:102A7000DD2454010894A108B1083CC0EE24FF24D1
:102A8000CA14DB041CF491E0E92EF12CDE010D9058
:102A90000020E9F71197AC1BBD0BF80180819181F3
:102AA000FC0101900020E9F73197E81BF90BAE0F0C
:102AB000BF1F1196AE0DBF1DCE01BD010E94F63A9B
:102AC000009731F4CE010E949E3AC0E0D0E015C0DC
:102AD000EC01F801608171810E945E3DEF2829F0D0
:102AE000CE0160E070E20E945E3D0894C11CD11CE2
:102AF0000E5F1F4FC814D9040CF2CE01DF91CF91A5
:102B00001F910F91FF90EF90DF90CF90BF90AF900B
:102B10009F908F900895CF92DF92EF92FF920F9344
:102B20001F93DF93CF93CDB7DEB78E01005F1F4FAA
:102B300080EA90E00E94F139D82EC92E60EA70E058
:102B40004E855F8598010E941A3E7C0197FF05C063
:102B50002DEFE22E2FEFF22E1DC08D2D9C2D9C010E
:102B6000890110C00F5F1F4F772767FD7095AC85F7
:102B7000BD851696ED91FC91179718968D919C91B5
:102B800019971995F8016081662361F78D2D9C2DA9
:102B90000E949E3AC701CF91DF911F910F91FF9044
:102BA000EF90DF90CF900895EF92FF920F931F93D5
:102BB000CF93DF938C01DC011296CD91DC911397BA
:102BC00033E0E32E30E2F32E24C0288139818C815A
:102BD0009D81009711F482E090E2EDB7FEB738973F
:102BE000EDBFFEBF3196ADB7BEB711960D931C93E6
:102BF0001297E282F38224833583868397830E942F
:102C00008B150884D985C02DEDB7FEB73896EDBF7A
:102C1000FEBF2097D1F6DF91CF911F910F91FF90CA
:102C2000EF9008958F929F92AF92BF92CF92DF92D2
:102C3000EF92FF920F931F93CF93DF938C016B0161
:102C40005A01922E832E6115710511F181E090E0F9
:102C50006EE270E00E94D539EC017C010097E9F149
:102C60000115110511F40EE010E20C831D8380E5BF
:102C700090E08C879D8781E090E060E570E00E94A5
:102C8000D5398A879B87009731F4CE010E949E3AFE
:102C9000EE24FF2422C0988A898ACE82DF82A88609
:102CA000B98690FC1AC000D000D0EDB7FEB73196BF
:102CB000ADB7BEB71196CD93DC93129780E190E249
:102CC000828393838C819D81848395830E948B155D
:102CD0008DB79EB706968DBF9EBFC701DF91CF917E
:102CE0001F910F91FF90EF90DF90CF90BF90AF902A
:102CF0009F908F9008952F923F924F925F926F9284
:102D00007F928F929F92AF92BF92CF92DF92EF927B
:102D1000FF920F931F93DF93CF93CDB7DEB7C155CB
:102D2000D040CDBFDEBF1C01142F052F62962FAF00
:102D30006297832E2DB73EB7285030402DBF3EBF3F
:102D4000EDB7FEB73196ADB7BEB711968D939C9394
:102D5000129784E190E28283938364837583629601
:102D6000BFAD6297B68387820E948B15212F302FCB
:102D7000C9012C0166247724EDB7FEB7389693C0BD
:102D80005301720100E010E081E090E08C0F9D1F84
:102D9000800F911FAC14BD0428F52DB73EB7285005
:102DA00030402DBF3EBFEDB7FEB73196ADB7BEB7D1
:102DB00011968D939C93129780E590E0801B910B68
:102DC000828393832BE230E224833583D7018C9175
:102DD000868317820E94C53DEDB7FEB73896EDBFDA
:102DE000FEBF04C061E370E20E94723D0D5F1F4FA1
:102DF0000894A11CB11C0894E11CF11C00331105BE
:102E000019F6CE01C19665E370E20E94723D52014F
:102E1000EE24FF248E010F5C1F4FC701860D971D06
:102E20008C159D05A0F4D5019C90892D992787FDCF
:102E300090950E94213D98012F5F3F4F892B19F0FB
:102E4000F801908203C0EEE2D801EC938901089466
:102E5000E11CF11C0894A11CB11CF0E1EF16F10477
:102E6000E1F6D8011C9200D000D0EDB7FEB7319644
:102E7000ADB7BEB711962D923C92129728E330E27F
:102E80002283338381E090E08C0F9D1F84839583A0
:102E90000E948B15A0E1B0E06A0E7B1E4A0E5B1EFD
:102EA000EDB7FEB73696EDBFFEBF6296CFAC629728
:102EB000D82C6C147D0408F463CFCF5ADF4FCDBFFC
:102EC000DEBFCF91DF911F910F91FF90EF90DF90C8
:102ED000CF90BF90AF909F908F907F906F905F90BA
:102EE0004F903F902F9008951F93CF93DF93EC0165
:102EF000162F6A3029F16D3019F18E859F85683063
:102F000009F0B1C0892B09F4E0C0888981FD14C0A3
:102F100000D00F92ADB7BEB71196CD93DC93129748
:102F20008FE390E213968D939C9314970E948B15D8
:102F30000F900F900F900F908E859F850197C3C0C3
:102F4000EA85FB858E859F85E80FF91F10828889A9
:102F500081FD10C000D00F92EDB7FEB7C183D283C0
:102F600083E490E2838394830E948B150F900F90EB
:102F70000F900F908A859B851A8A1B8A22E030E287
:102F80002C8B3D8B11C08A899B890A96FC01EE0F20
:102F9000FF1FEC0FFD1F2083318309978A8B9B8BCA
:102FA0000C9749F080E090E060E070E20E94493DBB
:102FB0009C01009741F76C897D89CE010E94BD1468
:102FC000FC01009721F4ECA5FDA5309779F08681EE
:102FD0009781888399836A897B89AE014C5E5F4FB4
:102FE0000280F381E02DCE0119951DC0AC89BD8909
:102FF0008C918823C1F000D000D02DB73EB72F5F51
:103000003F4FEDB7FEB7C183D28386E490E2F9016A
:1030100082839383A483B5830E948B158DB79EB75B
:1030200006968DBF9EBF1E861F86888980FD4DC077
:1030300000D000D0EDB7FEB73196ADB7BEB7119650
:10304000CD93DC93129780E190E2828393838C810D
:103050009D81848395830E948B15EDB7FEB73696CC
:10306000EDBFFEBF32C08F3491057CF5862F8052B4
:103070008F3558F5888981FD1CC000D000D0EDB790
:10308000FEB73196ADB7BEB71196CD93DC931297CC
:103090008DE590E282839383862F992787FD909513
:1030A000848395830E948B15EDB7FEB73696EDBFEE
:1030B000FEBFEA85FB858E859F85E80FF91F10838B
:1030C0008E859F8501968E879F87DF91CF911F9177
:1030D0000895CF92DF92EF92FF920F931F93DF93A9
:1030E000CF93CDB7DEB78E01045F1F4FF801E1909B
:1030F000F1908F0180EA90E00E94F139D82EC92E1C
:1031000060EA70E0A70198010E941A3E7C0197FDD9
:1031100005C08D2D9C2D9C0189010DC08D2D9C2DF0
:103120000E949E3A8DEFE82E8FEFF82E0CC00F5FB5
:103130001F4F0E940032F80180818823C1F78D2D36
:103140009C2D0E949E3AC701CF91DF911F910F9154
:10315000FF90EF90DF90CF9008952F923F924F9283
:103160005F926F927F928F929F92AF92BF92CF9217
:10317000DF92EF92FF920F931F93DF93CF93CDB720
:10318000DEB7C155D040CDBFDEBF162F072F6296E8
:103190004FAF6297852E00D000D0EDB7FEB73196C5
:1031A0002CE730E2ADB7BEB711962D933C93129742
:1031B000828393836296BFAD6297B48355830E94E6
:1031C0006918212F302FC9012C0166247724EDB70F
:1031D000FEB73696EDBFFEBF91E3292E312C2C0EA3
:1031E0003D1E8AC05301720100E010E081E090E0D2
:1031F0008C0F9D1F800F911FAC14BD0428F52DB7B7
:103200003EB7285030402DBF3EBFEDB7FEB73196D8
:10321000ADB7BEB711968D939C93129780E590E061
:10322000801B910B8283938323E930E224833583CF
:10323000D7018C91868317820E94C53DEDB7FEB7FA
:103240003896EDBFFEBF04C069E970E20E94723D8E
:103250000D5F1F4F0894A11CB11C0894E11CF11CC8
:103260000033110519F6C1016DE970E20E94723D4B
:1032700052018101EE24FF24C701860D971D8C1594
:103280009D05A0F4D5019C90892D992787FD9095E7
:103290000E94213D98012F5F3F4F892B19F0F801C3
:1032A000908203C0EEE2D801EC9389010894E11CFE
:1032B000F11C0894A11CB11CF0E1EF16F104E1F639
:1032C000D8011C9200D00F9220EA30E2EDB7FEB791
:1032D0002183328381E090E08C0F9D1F8383948350
:1032E0000E946918A0E1B0E06A0E7B1E4A0E5B1EC8
:1032F0000F900F900F900F906296CFAC6297D82CE2
:103300006C147D0408F46ECFCF5ADF4FCDBFDEBF03
:10331000CF91DF911F910F91FF90EF90DF90CF90B1
:10332000BF90AF909F908F907F906F905F904F90E5
:103330003F902F90089597FD03C027EA30E27EC0AA
:10334000FC017696E631F10508F04AC0E650FF4FE1
:10335000EE0FFF1F0590F491E02D19942FEA30E253
:103360006DC022EC30E26AC022ED30E267C028EE88
:1033700030E264C026EF30E261C024E031E25EC09A
:1033800022E131E25BC021E231E258C023E331E2C5
:1033900055C021E431E252C029E531E24FC026E6B2
:1033A00031E24CC02FE631E249C02BE731E246C0A2
:1033B00020E831E243C029E831E240C028E931E2A7
:1033C0003DC020EA31E23AC028EA31E237C02BEBB7
:1033D00031E234C026EC31E231C02EEC31E22EC0B5
:1033E0000F920F928DED91E2ADB7BEB711968D930E
:1033F0009C9312970E94691800D000D0EDB7FEB7D9
:10340000319688EF91E2ADB7BEB711968D939C933C
:1034100012978AE092E28283938388E390E0848328
:10342000958386EA9BE2868397830E94691821E34D
:1034300032E2EDB7FEB73896EDBFFEBFC901089581
:103440009C01E091F42BF091F52B82819381D901BD
:1034500018968D939C93199784819581FC016E9F9A
:10346000C0016F9F900D7E9F900D112468EE73E058
:103470000E948C39D9011A966D937C931B971696EE
:103480008D919C9117978E7F16968D939C9317978D
:103490000895E091F42BF091F52B22813381648122
:1034A000758188EE93E0AC01249FC001259F900DAB
:1034B000349F900D11240E948C39CB010895E09126
:1034C000F42BF091F52B309729F0828193810196AE
:1034D000828393830895CF93DF93C091F42BD0918F
:1034E000F52BEA81FB812C813D81AC01429FC0011B
:1034F000439F900D529F900D112468EE73E00E943F
:103500008C396E0F7F1F8A819B8186179707D8F3AE
:10351000DF91CF9108959C018617970748F4CB015E
:10352000821B930B4817590718F421E030E012C0B2
:103530006217730718F020E030E00CC080E090E0E4
:1035400020953095260F371F4217530710F481E05E
:1035500090E09C01C90108956817790730F49C0137
:1035600020953095260F371F03C09B01281B390B70
:10357000C9010895EF92FF920F931F93CF93DF93AA
:10358000E091F42BF091F52B868197818160868301
:103590009783C081D18108EE13E045C06E817F81A1
:1035A00060FD3EC028853985E091F42BF091F52B24
:1035B00042815381EA85FB852417350730F4CA011F
:1035C000821B930BE817F90750F04217530740F599
:1035D00020953095240F351FE217F30708F5616039
:1035E0006E837F836C817D81EA81FB81CE01199599
:1035F0008E8181FF15C08A859B85E091F42BF09127
:10360000F52B648175819C01209FC001219F900D45
:10361000309F900D11240E948C39CE010E94201AF7
:103620000990D881C02D209709F0B8CFE091F42BF4
:10363000F091F52B868197818E7F86839783C08159
:10364000D181EE24FF2423C08E8182FF1BC0E114B0
:10365000F10449F4E091F42BF091F52BA081B181B4
:103660008D919C9103C088819981F701808391831A
:1036700018810981CE010E949E3A212F302FC90165
:10368000EC0105C07E01888199819C01E9012097A8
:10369000D9F6DF91CF911F910F91FF90EF90089590
:1036A000CF93DF93EC010097E9F18E8182FF2CC06C
:1036B0000F920F9289E392E2ADB7BEB711968D9348
:1036C0009C9312970E94691800D000D0EDB7FEB706
:1036D000319684E592E2ADB7BEB711968D939C9377
:1036E000129780E892E2828393838AE690E0848353
:1036F000958380EB9BE2868397830E946918EDB7E0
:10370000FEB73896EDBFFEBFA091F42BB091F52B1C
:1037100016968C91169780FF08C08E819F818460D9
:103720008E839F8320E030E023C04D915C91119700
:103730009A01E0E0F0E017C02C173D0781F43097C4
:1037400031F4FA01808191818D939C9304C088812A
:10375000998180839183CE010E949E3AE3CFF90143
:10376000808191819C012115310531F72EEF3FEFCA
:10377000C901DF91CF910895AF92BF92CF92DF92AE
:10378000EF92FF920F931F93CF93DF935C016B0136
:10379000EA0179014115510519F400E010E035C046
:1037A00081E090E06CE070E00E94D539DC018C0192
:1037B000009759F11296CD93DC9313971496ED92DE
:1037C000FC921597CD2849F016968D919C911797EC
:1037D000826016968D939C931797C091F42BD0918D
:1037E000F52BE881F981309719F4A883B98309C0D2
:1037F000CF010190F081E02D3097D1F7FC01A0833B
:10380000B183CD01B5010E94201AC801DF91CF918B
:103810001F910F91FF90EF90DF90CF90BF90AF90EE
:103820000895CF93DF93EC01009719F42EEF3FEF4B
:1038300014C081E090E068E070E00E94D539FC019E
:103840008093F42B9093F52B009719F42DEF3FEF15
:1038500004C0C483D58320E030E0C901DF91CF915B
:1038600008958F929F92AF92BF92CF92DF92EF9284
:10387000FF920F931F93CF93DF934A015B01EC01FB
:1038800088E0C03AD807D1F4403895E2590790E073
:10389000690790E0790709F05AC02830310509F02E
:1038A00056C081E0E816F10409F051C0012B09F07F
:1038B0004EC0CD2809F04BC083E02AC0CD2809F0C6
:1038C00046C027303105A1F02830310520F42630DC
:1038D000310561F407C02830310531F02930310558
:1038E00029F408C081E007C083E005C080E003C080
:1038F00082E001C087E00130110539F00130110587
:1039000038F00230110519F502C0806201C08063F1
:1039100092E0E916F10409F488601C828D8384E04A
:10392000880C991CAA1CBB1C8A95D1F760E078E42E
:1039300088EE91E0A50194010E94B33921503040F6
:103940002E833F8388E18C8320E030E002C026EFA5
:103950003FEFC901DF91CF911F910F91FF90EF9041
:10396000DF90CF90BF90AF909F908F900895FC0113
:10397000818185FFFDCF6083E05AF84071F480912A
:10398000A10886FFFCCF8091A1088064E0EAF8E0FE
:10399000818388EE93E00197F1F70895EF92FF920B
:1039A0000F931F93CF93DF937C0120E030E000EA78
:1039B00018E0C8EED3E020C0FB01E20FF31FE08166
:1039C000D70111968C91119785FFFBCF8E2F9927E8
:1039D00087FD90958C93A05AB84061F48091A1081E
:1039E00086FFFCCF8091A1088064F8018183CE011D
:1039F0000197F1F72F5F3F4F24173507ECF2CA010B
:103A0000DF91CF911F910F91FF90EF900895FC01EE
:103A1000218130E020783070C9010895823091050D
:103A2000A1F08330910528F4009761F00197B1F47B
:103A300006C08330910561F0049781F40CC029EA37
:103A400032E23AC02BEA32E237C02DEA32E234C029
:103A50002FEA32E231C021EB32E22EC00F920F92F8
:103A600083EB92E2ADB7BEB711968D939C931297FC
:103A70000E94691800D000D0EDB7FEB731968EECE9
:103A800092E2ADB7BEB711968D939C93129780EEDC
:103A900092E2828393838EEA90E0848395838EEB17
:103AA0009BE2868397830E9469182EE033E2EDB78C
:103AB000FEB73896EDBFFEBFC9010895EF92FF92A1
:103AC0000F931F93182F092F7B010E94491AE12F92
:103AD000F02FEF2819F006EF1FEF06C0818187FF56
:103AE000FDCF8081082F10E0C8011F910F91FF903A
:103AF000EF900895CF92DF92EF92FF920F931F9372
:103B0000CF93DF936C017B018A01C0E0D0E00AC053
:103B1000C60160E070E00E945E1DF701EC0FFD1F22
:103B200080832196C017D1079CF3C801DF91CF9104
:103B30001F910F91FF90EF90DF90CF90089580E05C
:103B400090E008959C01883091054CF481E090E06C
:103B500002C0880F991F2A95E2F78093870608957F
:103B600087E0E0EAF0E082830E94E8070E942008F4
:103B700083E090E060E10E94D30784E090E060E1A0
:103B80000E94D307789480E090E00895EF92FF922E
:103B90000F931F93CF93DF938C01FA01623071056D
:103BA000BCF18281938163E47EE1A8010E94890FC8
:103BB000EC0197FF05C09FE0E92E93E2F92E04C0C7
:103BC00083E1E82E83E2F82ECE010E949B192DB7E7
:103BD0003EB72A5030402DBF3EBFEDB7FEB73196FD
:103BE000ADB7BEB711960D931C93129726E133E241
:103BF00022833383E482F582C683D78380879187CB
:103C00000E948B15EDB7FEB73A96EDBFFEBF14C00C
:103C100000D00F92ADB7BEB711968D939C931297BB
:103C200083E293E213968D939C9314970E948B15D5
:103C30000F900F900F900F90DF91CF911F910F91E8
:103C4000FF90EF9008952DB73EB7285030402DBF1C
:103C50003EBFEDB7FEB73196ADB7BEB711968D93A7
:103C60009C93129785E493E28283938364837583A4
:103C7000468357830E948B152DB73EB7285F3F4F71
:103C80002DBF3EBF08950F931F93182F092F611565
:103C90007105A9F400D00F92EDB7FEB73196ADB71C
:103CA000BEB711968C93918386E693E282839383C9
:103CB0000E948B150F900F900F900F901AC0CB01A0
:103CC0000E94FD1300D000D0EDB7FEB73196ADB71E
:103CD000BEB711961C93018322E833E2228333831B
:103CE000848395830E948B158DB79EB706968DBFF2
:103CF0009EBF1F910F910895CF92DF92EF92FF9296
:103D00000F931F93DF93CF9300D000D0CDB7DEB7D2
:103D10006C01FA01623071050CF457C00281138105
:103D2000C801BE016F5F7F4F40E050E00E94D23B70
:103D30009B01AC0189819A818017910709F05AC0D3
:103D400044C033E1E32E33E2F32EC8010E949B19F5
:103D50002DB73EB72A5030402DBF3EBFEDB7FEB75E
:103D60003196ADB7BEB71196CD92DC92129724E989
:103D700033E222833383E482F582068317838087CC
:103D800091870E948B15EDB7FEB73A96EDBFFEBF47
:103D9000CE0103960E94FD1300D000D0EDB7FEB710
:103DA0003196ADB7BEB71196CD92DC92129720EA4C
:103DB00033E222833383848395830E948B15EDB78E
:103DC000FEB73696EDBFFEBF23C000D00F92ADB751
:103DD000BEB71196CD92DC9212978AEA93E21396BF
:103DE0008D939C9314970E948B150F900F900F90BA
:103DF0000F900EC0C901BE016D5F7F4F0E94AA0BDC
:103E00008C0197FF9ECF2FE0E22E23E2F22E9DCF72
:103E10002696CDBFDEBFCF91DF911F910F91FF900E
:103E2000EF90DF90CF9008952F923F924F925F9244
:103E30006F927F928F929F92AF92BF92CF92DF92BA
:103E4000EF92FF920F931F93DF93CF93CDB7DEB71F
:103E50002A97CDBFDEBF3C016B017A01643071054A
:103E60000CF4DAC0DA0112960D911C911397C80177
:103E70005E010894A11CB11CB50140E050E00E9415
:103E8000D23B6F83788789819A818017910709F0E7
:103E9000D8C0C2C0F70106811781C801B50140E052
:103EA00050E00E94D23B9B01AC0189819A8180172E
:103EB000910709F4B1C0122F032F37FDADC028E0E0
:103EC00030E0E20EF31EC6010497B7010E941A15F6
:103ED0004C01009709F476C019870A87DC010D9020
:103EE0000020E9F77D010894E108F108E81AF90AD1
:103EF000C2010E94FD13EDB7FEB73A97EDBFFEBFBA
:103F00003196ADB7BEB711966D927C92129729EC9F
:103F100033E222833383E482F5828683978310879A
:103F200001870E948B15AA24BB24EDB7FEB73A96F1
:103F3000EDBFFEBF120175EE472E73E2572E35C05E
:103F40006701CA18DB08B4016A0D7B1D8F81988553
:103F5000A601910109851A850E94D7098C0197FF56
:103F600004C0C4010E949E3A2FC02DB73EB728500E
:103F700030402DBF3EBFEDB7FEB73196ADB7BEB7EF
:103F800011966D927C92129742825382848395831C
:103F9000C81AD90AC682D7820E948B15A00EB11EFC
:103FA000EDB7FEB73896EDBFFEBFAE14BF0444F2C6
:103FB000C4010E949E3A63E1E62E63E2F62E00E021
:103FC00010E006C00DEF1FEF5FE0E52E53E2F52E87
:103FD000C8010E949B192DB73EB72A5030402DBF13
:103FE0003EBFEDB7FEB73196ADB7BEB711966D9235
:103FF0007C92129726E133E222833383E482F582B6
:1040000006831783808791870E948B15EDB7FEB7D3
:104010003A96EDBFFEBF23C000D00F92ADB7BEB73A
:1040200011966D927C9212978AEF93E213968D937C
:104030009C9314970E948B150F900F900F900F90E8
:104040000EC043E0442E512C4C0E5D1EF7018481BE
:104050009581B2010E945012892BF1F21BCF2A9652
:10406000CDBFDEBFCF91DF911F910F91FF90EF90F9
:10407000DF90CF90BF90AF909F908F907F906F9088
:104080005F904F903F902F9008952F923F924F92C4
:104090005F926F927F928F929F92AF92BF92CF92D8
:1040A000DF92EF92FF920F931F93DF93CF930F92C4
:1040B0000F92CDB7DEB73C016B017A016330710519
:1040C0000CF4A6C0DA0112960D911C911397C80149
:1040D000BE016F5F7F4F40E050E00E94D23B1B016A
:1040E00089819A818017910709F0A7C091C0D401F6
:1040F0000D900020E9F77D010894E108F108E81827
:10410000F90800D000D0EDB7FEB73196ADB7BEB715
:1041100011966D927C9212978AE294E28283938345
:10412000E482F5820E948B15AA24BB24EDB7FEB76A
:104130003696EDBFFEBFA5EE4A2EA3E25A2E31C041
:104140006701CA18DB08B4016A0D7B1DC101A60115
:104150000E94DE0B8C0197FF04C0C4010E949E3AAE
:104160002FC02DB73EB7285030402DBF3EBFEDB712
:10417000FEB73196ADB7BEB711966D927C9212978D
:104180004282538284839583C81AD90AC682D78211
:104190000E948B15A00EB11EEDB7FEB73896EDBF8D
:1041A000FEBFAE14BF0464F2C4010E949E3AF3E164
:1041B000EF2EF3E2FF2E00E010E006C00DEF1FEF40
:1041C000EFE0EE2EE3E2FE2EC8010E949B192DB710
:1041D0003EB72A5030402DBF3EBFEDB7FEB73196F7
:1041E000ADB7BEB711966D927C92129726E133E27D
:1041F00022833383E482F582068317838087918745
:104200000E948B15EDB7FEB73A96EDBFFEBF23C0F7
:1042100000D00F92ADB7BEB711966D927C921297F7
:104220008DE394E213968D939C9314970E948B15C3
:104230000F900F900F900F900EC0E4E0F0E0EE0EA4
:10424000FF1EC6010297B7010E941A154C01009784
:1042500009F04DCFB3CF0F900F90CF91DF911F9109
:104260000F91FF90EF90DF90CF90BF90AF909F9015
:104270008F907F906F905F904F903F902F90089518
:10428000CF92DF92EF92FF920F931F93DF93CF9322
:104290000F920F92CDB7DEB76C01FA016230710553
:1042A000D4F102811381C801BE016F5F7F4F40E0EE
:1042B00050E00E94D23B9B01AC0189819A8180171A
:1042C0009107F1F528C083E1E82E83E2F82EC801BA
:1042D0000E949B192DB73EB72A5030402DBF3EBFDC
:1042E000EDB7FEB73196ADB7BEB71196CD92DC9261
:1042F000129726E133E222833383E482F582068338
:104300001783808791870E948B15EDB7FEB73A9689
:10431000EDBFFEBF20C000D00F92ADB7BEB7119663
:10432000CD92DC9212978FE594E213968D939C9335
:1043300014970E948B150F900F900F900F900BC049
:10434000C9010E94200F8C0197FFBDCFBFE0EB2E6B
:10435000B3E2FB2EBCCF0F900F90CF91DF911F9156
:104360000F91FF90EF90DF90CF9008954F925F9262
:104370006F927F928F929F92AF92BF92CF92DF9275
:10438000EF92FF920F931F93DF93CF9300D000D053
:10439000CDB7DEB74C017A01643071050CF464C00E
:1043A000DA0112960D911C911397C8013E010894F1
:1043B000611C711CB30140E050E00E94D23B5B01E4
:1043C0006C0189819A818017910709F062C04CC005
:1043D000F70106811781C801B30140E050E00E9457
:1043E000D23B9B01AC0189819A8180179107E1F151
:1043F00037FD3AC0C501B201A90123E23EE10BE657
:1044000012E274010E946C0C8C0197FF05C03FE022
:10441000E32E33E2F32E04C023E1E22E23E2F22E58
:10442000C8010E949B192DB73EB72A5030402DBFBE
:104430003EBFEDB7FEB73196ADB7BEB711968D92C0
:104440009C92129726E133E222833383E482F58241
:1044500006831783808791870E948B15EDB7FEB77F
:104460003A96EDBFFEBF23C000D00F92ADB7BEB7E6
:1044700011968D929C92129787E794E213968D93F2
:104480009C9314970E948B150F900F900F900F9094
:104490000EC093E0492E512C4C0E5D1EF701848115
:1044A0009581B2010E945012892BF1F291CF26968C
:1044B000CDBFDEBFCF91DF911F910F91FF90EF90A5
:1044C000DF90CF90BF90AF909F908F907F906F9034
:1044D0005F904F900895AF92BF92CF92DF92EF928C
:1044E000FF920F931F93DF93CF93CDB7DEB7C054E6
:1044F000D040CDBFDEBF5C017B018A014115510573
:1045000019F42DE934E202C02FEA34E28DB79EB7E8
:104510000A978DBF9EBFEDB7FEB73196ADB7BEB758
:104520001196AC92B18280EB94E282839383E48211
:10453000F58206831783208731870E948B158DB7FC
:104540009EB70A968DBF9EBF6E010894C11CD11CF8
:1045500017C00134110510F4A80102C040E450E076
:10456000C701B6010E94250C9C01181619068CF78C
:10457000081B190BC5016CEC74E2A6010E947B16A6
:104580001016110634F3C05CDF4FCDBFDEBFCF91F4
:10459000DF911F910F91FF90EF90DF90CF90BF9030
:1045A000AF9008954F925F926F927F928F929F92F9
:1045B000AF92BF92CF92DF92EF92FF920F931F9331
:1045C000DF93CF930F920F92CDB7DEB73C015B0123
:1045D0004A01623071050CF45FC0DA0112960D9148
:1045E0001C911397C8012E010894411C511CB20163
:1045F00040E050E00E94D23B6B017C0189819A81AE
:104600008017910709F05DC047C0F401048115814E
:10461000C801B20140E050E00E94D23B9B01AC01D6
:1046200089819A8180179107B9F1B901C6014CE7D8
:1046300053E293010E94E10C8C0197FF05C05FE0FB
:10464000E52E53E2F52E04C043E1E42E43E2F42EBE
:10465000C8010E949B192DB73EB72A5030402DBF8C
:104660003EBFEDB7FEB73196ADB7BEB711966D92AE
:104670007C92129726E133E222833383E482F5822F
:1046800006831783808791870E948B15EDB7FEB74D
:104690003A96EDBFFEBF1DC000D00F92ADB7BEB7BA
:1046A00011966D927C9212978FEC94E213968D93F3
:1046B0009C9314970E948B150F900F900F900F9062
:1046C00008C0B2E0AB16B10409F09FCF61E070E022
:1046D000ADCF0F900F90CF91DF911F910F91FF9071
:1046E000EF90DF90CF90BF90AF909F908F907F9092
:1046F0006F905F904F900895EF92FF920F931F93EA
:10470000CF93DF93F82EE92E8B0100D000D0EDB7C8
:10471000FEB73196ADB7BEB711968C93918382EFF9
:1047200094E282839383648375830E948B152DB7F3
:104730003EB72A5F3F4F2DBF3EBFC80163E27EE117
:104740004BE652E22F2D3E2D0E94E00FEC0197FF29
:1047500003C00FE013E202C003E113E2CE010E94A6
:104760009B19ADB7BEB71A97ADBFBEBFEDB7FEB7C9
:1047700031961196FC92E18226E133E22283338363
:1047800004831583C683D783808791870E948B1506
:104790002DB73EB7265F3F4F2DBF3EBFDF91CF9174
:1047A0001F910F91FF90EF9008954F925F926F923B
:1047B0007F928F929F92AF92BF92CF92DF92EF92B1
:1047C000FF920F931F93DF93CF9300D000D0CDB70C
:1047D000DEB72C017A01643071050CF45FC0DA0198
:1047E00012960D911C911397C8014E010894811CDB
:1047F000911CB40140E050E00E94D23B5B016C018F
:1048000089819A818017910709F05DC047C0F7013F
:1048100006811781C801B40140E050E00E94D23BFC
:104820009B01AC0189819A8180179107B9F137FD0D
:1048300035C0C501B301A9010E94200D8C0197FF6D
:1048400005C0EFE0EE2EE3E2FE2E04C073E1E72E9A
:1048500073E2F72EC8010E949B192DB73EB72A506C
:1048600030402DBF3EBFEDB7FEB73196ADB7BEB7F6
:1048700011964D925C92129726E133E222833383A4
:10488000E482F58206831783808791870E948B15C7
:10489000EDB7FEB73A96EDBFFEBF23C000D00F9232
:1048A000ADB7BEB711964D925C92129786E195E234
:1048B00013968D939C9314970E948B150F900F90D5
:1048C0000F900F900EC063E0662E712C6C0E7D1E53
:1048D000F70184819581B3010E945012892BF1F276
:1048E00096CF2696CDBFDEBFCF91DF911F910F915E
:1048F000FF90EF90DF90CF90BF90AF909F908F9000
:104900007F906F905F904F9008958F929F92AF929B
:10491000BF92CF92DF92EF92FF920F931F93DF939C
:10492000CF930F920F92CDB7DEB74C016B015A01B6
:10493000623071050CF472C0DA0112960D911C916F
:104940001397C80169E375E20E94693D009719F465
:10495000EE24FF2416C0C80160E475E20E94693DA0
:10496000009721F411E0E12EF12C0BC0C80166E4A0
:1049700075E20E94693D009709F050C0B2E0EB2E4D
:10498000F12CB2E0CB16D10419F460E070E013C052
:10499000F50104811581C801BE016F5F7F4F40E0C2
:1049A00050E00E94D23B9B01AC0189819A81801723
:1049B0009107A1F1B901C7010E945B108C0197FF1B
:1049C00005C0AFE0EA2EA3E2FA2E04C0F3E1EF2E19
:1049D000F3E2FF2EC8010E949B192DB73EB72A5063
:1049E00030402DBF3EBFEDB7FEB73196ADB7BEB775
:1049F00011968D929C92129726E133E222833383A3
:104A0000E482F58206831783808791870E948B1545
:104A1000EDB7FEB73A96EDBFFEBF14C000D00F92BF
:104A2000ADB7BEB711968D929C9212978AE495E22B
:104A300013968D939C9314970E948B150F900F9053
:104A40000F900F900F900F90CF91DF911F910F91CA
:104A5000FF90EF90DF90CF90BF90AF909F908F909E
:104A600008950F931F93DF93CF930F920F92CDB7BB
:104A7000DEB78C01CE0101960E94DC0AAC0197FFE3
:104A800003C02FE033E202C023E133E28DB79EB7CB
:104A90000A978DBF9EBFEDB7FEB73196ADB7BEB7D3
:104AA00011960D931C93129788E795E28283938366
:104AB000248335834683578389819A8180879187B0
:104AC0000E948B158DB79EB70A968DBF9EBF0F9023
:104AD0000F90CF91DF911F910F910895CF92DF92A8
:104AE000EF92FF920F931F93DF93CF930F920F924A
:104AF000CDB7DEB76C01FA0162307105D4F10281E5
:104B00001381C801BE016F5F7F4F40E050E00E94FB
:104B1000D23B9B01AC0189819A8180179107F1F505
:104B200028C093E1E92E93E2F92EC8010E949B1957
:104B30002DB73EB72A5030402DBF3EBFEDB7FEB770
:104B40003196ADB7BEB71196CD92DC92129726E1A1
:104B500033E222833383E482F582068317838087DE
:104B600091870E948B15EDB7FEB73A96EDBFFEBF59
:104B700020C000D00F92ADB7BEB71196CD92DC9297
:104B800012978DE895E213968D939C9314970E944B
:104B90008B150F900F900F900F900BC0C9010E94C2
:104BA000730B8C0197FFBDCF8FE0E82E83E2F82EC8
:104BB000BCCF0F900F90CF91DF911F910F91FF907D
:104BC000EF90DF90CF9008950F931F93DF93CF93D3
:104BD000CDB7DEB76097CDBFDEBF8C01CE010196A9
:104BE000BE016B5F7F4FAE01475F5F4F9E01235F4A
:104BF0003F4F0E94F80AAC0197FF03C02FE033E259
:104C000002C023E133E28DB79EB708978DBF9EBFE8
:104C1000EDB7FEB73196ADB7BEB711960D931C93A5
:104C2000129785EA95E282839383248335834683B2
:104C300057830E948B158DB79EB708968DBF9EBF78
:104C4000CE0101960E94FD1300D000D0EDB7FEB753
:104C50003196ADB7BEB711960D931C9312972DEAFE
:104C600035E222833383848395830E948B158DB72D
:104C70009EB706968DBF9EBFCE0105960E94FD137E
:104C800000D000D0EDB7FEB73196ADB7BEB71196E4
:104C90000D931C93129724EB35E222833383848394
:104CA00095830E948B158DB79EB706968DBF9EBFCC
:104CB000CE0109960E94FD1300D000D0EDB7FEB7DB
:104CC0003196ADB7BEB711960D931C9312972DEB8D
:104CD00035E222833383848395830E948B158DB7BD
:104CE0009EB706968DBF9EBFCE010D960E94FD1306
:104CF00000D000D0EDB7FEB73196ADB7BEB7119674
:104D00000D931C93129724EC35E222833383848322
:104D100095830E948B158DB79EB706968DBF9EBF5B
:104D20006096CDBFDEBFCF91DF911F910F910895A7
:104D3000CF92DF92EF92FF920F931F93DF93CF9367
:104D4000CDB7DEB76097CDBFDEBF6C018B017A01B6
:104D500080919E2B90919F2BA091A02BB091A12B85
:104D60008D839E83AF83B88789879A87AB87BC87FB
:104D70008D879E87AF87B88B623071050CF475C044
:104D8000DA0112968D919C911397BE016F5F7F4F50
:104D90000E945012892B09F468C00230110541F1BC
:104DA000F70184819581BE016B5F7F4F0E94501295
:104DB000892B09F45AC003301105D1F0D70116969A
:104DC0008D919C911797BE01675F7F4F0E94501293
:104DD000892B09F44AC00530110554F0F70180858C
:104DE0009185BE01635F7F4F0E945012892BE9F1CC
:104DF000CE010196BE016B5F7F4FAE01475F5F4FF3
:104E00009E01235F3F4F0E94830B8C0197FF05C0DB
:104E10003FE0E32E33E2F32E04C023E1E22E23E24F
:104E2000F22EC8010E949B192DB73EB72A50304080
:104E30002DBF3EBFEDB7FEB73196ADB7BEB71196E9
:104E4000CD92DC92129726E133E222833383E4820F
:104E5000F58206831783808791870E948B15EDB7B3
:104E6000FEB73A96EDBFFEBF14C000D00F92ADB7AB
:104E7000BEB71196CD92DC9212978EEC95E2139606
:104E80008D939C9314970E948B150F900F900F9009
:104E90000F906096CDBFDEBFCF91DF911F910F9134
:104EA000FF90EF90DF90CF9008958F929F92AF92F6
:104EB000BF92CF92DF92EF92FF920F931F93DF93F7
:104EC000CF93CDB7DEB7C854D040CDBFDEBF5C01B5
:104ED0008E010E5D1F4FC8010E94BF106C0152E48D
:104EE000E52EF12CEC0EFD1ED7014C91CE01019662
:104EF000B80150E00E944E3DF701E080D7FE03C0AC
:104F00000FE013E202C003E113E2EE2029F04E01AC
:104F10000894811C911C04C049EF842E45E2942E14
:104F2000FE01ED5BFF4F2081FE01EC5BFF4F308106
:104F3000FE01EB5BFF4F4081FE01EA5BFF4F5081BA
:104F4000FE01E95BFF4F6081FE01E85BFF4F70816E
:104F5000FE01EE0DF11D11828DB79EB746978DBFF4
:104F60009EBFEDB7FEB73196ADB7BEB71196AD9205
:104F7000BC9212978DEF95E282839383048315830D
:104F8000C682D782808691862287138634871586CB
:104F900046871786508B118A628B138A748B158A09
:104FA0000E948B15EDB7FEB77696EDBFFEBFC85BCE
:104FB000DF4FCDBFDEBFCF91DF911F910F91FF90EB
:104FC000EF90DF90CF90BF90AF909F908F9008951B
:104FD000AC01DC010D900020E9F71197A81BB90B7B
:104FE000FB01A0A3CB01BA014A2F50E00E944E3D25
:104FF00081E090E008950F931F93DF93CF9300D04B
:1050000000D0CDB7DEB78C01CE0101960E94F8101A
:10501000AC0197FF03C02FE033E202C023E133E28B
:105020008DB79EB744978DBF9EBFEDB7FEB7319643
:10503000ADB7BEB711960D931C93129788E296E216
:105040008283938324833583468357838981808732
:1050500011868A81828713868B81848715868C814D
:10506000868717868D81808B118A8E81828B138A29
:105070000E948B158DB79EB744968DBF9EBF269616
:10508000CDBFDEBFCF91DF911F910F910895EF92B9
:10509000FF920F931F93CF93DF937C010E948C0BA1
:1050A000EC0197FF03C00FE013E202C003E113E23B
:1050B000CE010E949B192DB73EB72A5030402DBF1C
:1050C0003EBFEDB7FEB73196ADB7BEB71196ED92C4
:1050D000FC92129726E133E2228333830483158303
:1050E000C683D783808791870E948B152DB73EB7E3
:1050F000265F3F4F2DBF3EBFDF91CF911F910F9194
:10510000FF90EF900895AF92BF92CF92DF92EF920F
:10511000FF920F931F93DF93CF93CDB7DEB7A39783
:10512000CDBFDEBF5C017A01E3E0CE2ED12CCC0EE8
:10513000DD1E81E2D6011D928A95E9F76430710582
:10514000FCF0FA0182819381B6010E94E827892B45
:1051500009F471C0D70116960D911C911797C801DB
:10516000BE016F5F7F4F40E050E00E94D23B9B0149
:10517000AC0189819A818017910709F071C05BC0E9
:105180006330710581F4FA0182819381B6010E9436
:10519000E827892B09F44FC0D70114966D917C91B3
:1051A0001597C60114C06230710551F4FA0182816D
:1051B0009381B6010E94E827892BE9F1C60105C059
:1051C00061307105C1F580E090E060E070E040E0A2
:1051D00050E00E9428118C0197FF05C07FE0E72E68
:1051E00073E2F72E04C063E1E62E63E2F62EC801F7
:1051F0000E949B192DB73EB72A5030402DBF3EBFAD
:10520000EDB7FEB73196ADB7BEB71196AD92BC9271
:10521000129726E133E222833383E482F582068308
:105220001783808791870E948B15EDB7FEB73A965A
:10523000EDBFFEBF1BC000D00F92ADB7BEB7119639
:10524000AD92BC92129780E596E213968D939C9353
:1052500014970E948B150F900F900F900F9006C01F
:10526000F70164817581C601A901B3CFA396CDBFB3
:10527000DEBFCF91DF911F910F91FF90EF90DF90F4
:10528000CF90BF90AF9008954F925F926F927F92B0
:105290008F929F92AF92BF92CF92DF92EF92FF9246
:1052A0000F931F93CF93DF93582E492EEB013A01B2
:1052B0004801590100D00F92EDB7FEB73196ADB756
:1052C000BEB711968C9391838BE998E28283938386
:1052D0000E948B150F900F900F900F902097E1F088
:1052E000CE010E949B19EDB7FEB73897EDBFFEBF08
:1052F0003196ADB7BEB711965C9241822EE938E285
:1053000022833383C483D583868397830E948B153E
:10531000EDB7FEB738965BC081149104A104B104C7
:1053200009F440C06301EE24D7FCE094FE2C2DB7B5
:105330003EB7225130402DBF3EBF0DB71EB70F5FA5
:105340001F4FADB7BEB711965C92F801418281EB59
:1053500098E28283938364827582D80116968D9237
:105360009D92AD92BC921997C701B601A501940117
:105370000E94B339F8012287338744875587C701D4
:10538000B601A50194010E94B339D8011E966D9310
:105390007D938D939C9351970E948B15EDB7FEB72B
:1053A000729615C000D000D0EDB7FEB73196ADB7FC
:1053B000BEB711965C92418284EE98E28283938319
:1053C000648275820E948B15EDB7FEB73696EDBFED
:1053D000FEBFDF91CF911F910F91FF90EF90DF9073
:1053E000CF90BF90AF909F908F907F906F905F9085
:1053F0004F9008950F931F93CF93DF93182F092F8A
:10540000EB0100D00F92EDB7FEB73196ADB7BEB746
:1054100011968C9391838AE099E2828393830E9410
:105420008B150F900F900F900F901C161D06DCF43B
:10543000CE0160E570E00E94A039892BA1F400D074
:105440000F92EDB7FEB73196ADB7BEB711961C936C
:1054500001838BE998E2828393830E948B150F90DE
:105460000F900F900F90DF91CF911F910F910895A2
:10547000AF92BF92CF92DF92EF92FF920F931F9362
:10548000CF93DF93EC01B62EA72E88899989892BBB
:1054900071F08C819D812E813F81AC01429FC001C2
:1054A000439F900D529F900D11246C0104C0CA8837
:1054B000DB88EC88FD886C857D85888599850E94D0
:1054C000AC1AEA8DFB8D309749F08C0120E030E07A
:1054D0008C8D9D8D6B2D7A2DA60119958A819B81CE
:1054E0000E949E3A888199810E94200F888999891B
:1054F000892B21F48E899F890E94200FCE010E9462
:105500009E3A8B2D9A2DDF91CF911F910F91FF9095
:10551000EF90DF90CF90BF90AF9008958F929F92C1
:10552000AF92BF92CF92DF92EF92FF920F931F93B1
:10553000CF93DF934C017B016A01590181E090E038
:105540006EE170E00E94D539EC01009719F480E01B
:1055500090E010C0EC82FD82C88ED98EAA8EBB8EE0
:105560000C8F1D8FC7010E94F1398A839B8300979E
:1055700031F4CE016DEF7FEF0E94382A23C080E026
:1055800090E060E070E00E945B10BC01888399832A
:1055900097FD14C06EE97BE2A4010E94200DBC01BE
:1055A00097FD0CC08881998161E070E04FEE5AE26E
:1055B0009E010E94E10CBC0197FF02C0CE01DCCF2E
:1055C00088819981DF91CF911F910F91FF90EF908A
:1055D000DF90CF90BF90AF909F908F900895CF9322
:1055E000DF93EC01CB0164E57BE24DE05BE29E01E1
:1055F0000E94E00FBC018E8B9F8B97FF03C0CE01F2
:105600000E94382A0E94491AA0E0B0E08887998752
:10561000AA87BB87DF91CF910895CF93DF939B013A
:10562000EC0188899989892BE1F5452B61F40E9469
:10563000491AA0E0B0E08C879D87AE87BF87CE0176
:1056400060E070E00BC06A817B814C815D81C901A3
:105650000E94250CBC0197FF04C0CE010E94382A8D
:1056600020C0EE81FF813196EE83FF839C014427A9
:1056700037FD4095542F8A899B89AC89BD89820F5B
:10568000931FA41FB51F8A8B9B8BAC8BBD8B288D62
:10569000398D2115310529F08C8D9D8DBF01F901C2
:1056A0001995DF91CF9108954F925F926F927F92FB
:1056B0008F929F92AF92BF92CF92DF92EF92FF9222
:1056C0000F931F93CF93DF93EC01452B19F46CEFED
:1056D0007FEFA6C088899989892B61F50F920F9277
:1056E0008CE099E2ADB7BEB711968D939C9312975B
:1056F0000E94691800D000D0EDB7FEB7319687E25E
:1057000099E2ADB7BEB711968D939C93129782E440
:1057100099E28283938380EB90E0848395838DEC80
:105720009BE2868397830E946918EDB7FEB738968F
:10573000EDBFFEBF0E94491AA0E0B0E088879987BC
:10574000AA87BB87EE24FF244CE0442E49E2542E66
:1057500033E5632E39E2732E22E4822E29E2922E63
:105760009FE0A92E91E0B92E85EDC82E8BE2D82EB0
:1057700044C06A817B81600F711F401B510B88817F
:1057800099810E94DE0BBC0197FD2EC0080F191FE6
:105790004C815D810417150760F30417150709F4A0
:1057A00052C00F920F92ADB7BEB711964D925C9258
:1057B00012970E94691800D000D0EDB7FEB731965D
:1057C000ADB7BEB711966D927C921297828293828A
:1057D000A482B582C682D7820E946918EDB7FEB74F
:1057E0003896EDBFFEBF2FC0CE011AC08C8D9D8DA7
:1057F000B70119950894E11CF11C8E819F81E81670
:10580000F90618F400E010E0C3CF0E94491AA0E0A6
:10581000B0E08C879D87AE87BF87CE0160E070E0E7
:105820000E94382ADF91CF911F910F91FF90EF9046
:10583000DF90CF90BF90AF909F908F907F906F90B0
:105840005F904F900895E88DF98D309779F6D2CF1B
:105850004F925F926F927F928F929F92AF92BF9280
:10586000CF92DF92EF92FF920F931F93CF93DF932C
:105870002C013B014A0159014115510509F44CC065
:105880002115310509F448C06115710509F444C0BA
:1058900081E090E06EE170E00E94D539EC01009764
:1058A00019F42DEF3FEF3AC08E829F82AC82BD8209
:1058B000088F198FEA8EFB8ECC8EDD8E81E090E012
:1058C000888B998BC5010E94F1398A839B8300974D
:1058D00021F4CE016DEF7FEF18C080E090E060E032
:1058E00070E00E945B10BC018883998397FD0CC017
:1058F000B201A30124E53BE20DE01BE27E010E9420
:105900006C0CBC0197FF05C0CE010E94382A9C0197
:1059100005C02881398102C02EEF3FEFC901DF9118
:10592000CF911F910F91FF90EF90DF90CF90BF909C
:10593000AF909F908F907F906F905F904F90089561
:105940002F923F924F925F926F927F928F929F928F
:10595000AF92BF92CF92DF92EF92FF920F931F937D
:10596000DF93CF9300D000D0CDB7DEB75C013B0111
:105970006A0180919E2B90919F2BA091A02BB091BA
:10598000A12B89839A83AB83BC8301E010E038E8C4
:10599000832E33E1932E20E034E02D833E83412C8F
:1059A00024E0522E2224332470C0F801EE0FFF1F92
:1059B000EC0DFD1DE080F180C70167E779E20E94F0
:1059C000693D009789F40F5F1F4F061517050CF00E
:1059D000EEC0F801EE0FFF1FEC0DFD1D80819181DF
:1059E0000E94013D4C014FC0C7016AE779E20E9465
:1059F000693D009791F40F5F1F4F061517050CF0D6
:105A0000D6C0F801EE0FFF1FEC0DFD1D80819181C6
:105A10000E94013D8D839E8336C0C7016DE779E208
:105A20000E94693D009789F40F5F1F4F0615170507
:105A30000CF0BDC0F801EE0FFF1FEC0DFD1D8081C5
:105A400091810E94013D2C011EC0C70160E879E2EE
:105A50000E94693D009721F4F1E02F2E312C13C0F4
:105A6000C70163E879E20E94693D009719F4222496
:105A7000332409C0C701BE016F5F7F4F0E945012DF
:105A8000892B09F494C00F5F1F4F061517050CF4FE
:105A90008CCF21143104C9F089819A81AB81BC81FA
:105AA0000097A105B10509F482C0CE010196B401A9
:105AB0004D815E8192010AEF19E2E4E4EE2EE9E203
:105AC000FE2E65010E94282C09C0C401B2014AEFD4
:105AD00059E224E439E285010E948E2A8C0197FF65
:105AE0001BC00E949B19ADB7BEB71A97ADBFBEBF12
:105AF000EDB7FEB731961196AD92BC92129726E89B
:105B000039E22283338322E939E224833583068311
:105B100017838087918743C0232859F1CE010196CE
:105B20000E94FD132DB73EB72E5030402DBF3EBF13
:105B3000EDB7FEB73196ADB7BEB71196AD92BC9238
:105B4000129726E939E22283338384839583868200
:105B500097822D813E812087318742865386048734
:105B600015870E948B158DB79EB70E968DBF9EBF71
:105B700032C0ADB7BEB71A97ADBFBEBFEDB7FEB767
:105B800031961196AD92BC92129787EC99E282837E
:105B900093838482958246825782008711870E9470
:105BA0008B15EDB7FEB73A96EDBFFEBF14C000D01F
:105BB0000F92ADB7BEB71196AD92BC92129782EF1D
:105BC00099E213968D939C9314970E948B150F90D6
:105BD0000F900F900F902696CDBFDEBFCF91DF9133
:105BE0001F910F91FF90EF90DF90CF90BF90AF90FB
:105BF0009F908F907F906F905F904F903F902F90ED
:105C000008952F923F924F925F926F927F928F9260
:105C10009F92AF92BF92CF92DF92EF92FF920F933B
:105C20001F93DF93CF9300D00F92CDB7DEB75C0107
:105C30003B0129833A8328016115710519F48B838F
:105C40009C830BC0FB010190F081E02DE80FF91F50
:105C5000EB83FC83FB01108211828A018824992442
:105C600015010894211C311C50C0EB81FC819081EE
:105C7000992309F452C0F8018081C92EDD24C7FCA4
:105C8000D0944114510431F0E82EFF24E7FCF09445
:105C9000C60109C0992787FD90950E942F3D7C0180
:105CA000C6010E942F3DE816F90629F1F80180810E
:105CB000F501F0804114510449F0C82EDD24C7FCE1
:105CC000D0948F2D992787FD90950CC0992787FD3B
:105CD00090950E942F3D6C018F2D992787FD9095FF
:105CE0000E942F3DC816D90619F0AB82BC8208C0AD
:105CF0002B823C8205C08B819C8101968B839C8387
:105D00000F5F1F4F0894811C911CE981FA818E1648
:105D10009F0608F4AACF00E010E06114710439F086
:105D20008B819C818A199B09F30180839183C8012F
:105D30002496CDBFDEBFCF91DF911F910F91FF90D1
:105D4000EF90DF90CF90BF90AF909F908F907F901B
:105D50006F905F904F903F902F900895CF92DF9279
:105D6000EF92FF920F931F93CF93DF936C017B0110
:105D7000DB010D900020E9F78D0101501040061B5A
:105D8000170BC0E0D0E00EC0B7016C0F7D1FA8015B
:105D90004C1B5D0BC6010E94DE0B9C0197FD07C0EA
:105DA000C80FD91FC017D1077CF320E030E0C9012C
:105DB000DF91CF911F910F91FF90EF90DF90CF90E7
:105DC00008958F929F92AF92BF92CF92DF92EF92FF
:105DD000FF920F931F93CF93DF934C015B016A01F6
:105DE00080E091E00E94F139F82EE92E00E010E009
:105DF00021C0E601C01BD10B81E0C130D80714F0EF
:105E0000C0E0D1E0B501600F711F8F2D9E2DAE0156
:105E10000E94373DC4016F2D7E2DAE010E94DE0B26
:105E2000EC0197FF05C08F2D9E2D0E949E3A0BC05E
:105E3000080F191F0C151D05E4F28F2D9E2D0E94D1
:105E40009E3AC0E0D0E0CE01DF91CF911F910F913B
:105E5000FF90EF90DF90CF90BF90AF909F908F908A
:105E60000895EF92FF920F931F937C018B01CB015A
:105E70000E94403DAC01C701B8010E94E12E1F9174
:105E80000F91FF90EF900895EF92FF920F931F9361
:105E9000DF93CF93CDB7DEB7AC97CDBFDEBF7C012C
:105EA000009719F42FEF3FEFE2C08EE49FE2A1E4E8
:105EB000B0E08B8F9C8FAD8FBE8FFE017F968EE002
:105EC000DF011D928A95E9F7C70167E876E00E9435
:105ED000312F9C0197FDCBC08E010F5F1F4FC80172
:105EE00060E070E040E050E020E030E00E94F80A1E
:105EF000892B19F002E21AE204C0C8010E94FD13C6
:105F00008C01C70162E776E00E94312F9C0197FD6A
:105F1000AEC0C701B8010E94AE2E9C0197FDA7C07C
:105F2000C70167E576E00E94312F9C0197FD9FC075
:105F3000CE0105960E94F810892B99F52DB73EB732
:105F4000225130402DBF3EBFEDB7FEB73196CE0196
:105F50004B96ADB7BEB711968D939C93129782E185
:105F600090E08283938386E29AE2848395838D8195
:105F7000868317828E81808711868F818287138620
:105F80008885848715868985868717868A85808B8C
:105F9000118A0E94C53D2DB73EB72E5E3F4F2DBFE3
:105FA0003EBFC70161E476E00E94312F9C0197FD5E
:105FB0005EC0C701BE01655E7F4F0E94AE2E9C0190
:105FC00097FD55C0C70166E276E00E94312F9C0123
:105FD00097FD4DC0C70160E176E00E94312F9C0122
:105FE00097FD45C00E94BF33ADB7BEB71897ADBF90
:105FF000BEBFEDB7FEB731968E01055F1F4F1196FC
:106000000D931C93129720E130E02283338324E424
:106010003AE224833583868397830E94C53D2DB75A
:106020003EB7285F3F4F2DBF3EBFC701B8010E945A
:10603000AE2E9C0197FD1BC0C70165EF75E00E9465
:10604000312F9C0197FD13C0C70168EC73E00E94DB
:10605000312F9C0197FD0BC0C70160E272E00E94E6
:10606000312F9C011816190614F420E030E0C90104
:10607000AC96CDBFDEBFCF91DF911F910F91FF9006
:10608000EF900895EF92FF920F931F93DF93CF93BA
:106090000F920F92CDB7DEB78C017B0169E47AE2F3
:1060A0000E94693D009799F1C8016BE47AE20E9471
:1060B000693D009761F1C8016EE47AE24CE050E07E
:1060C0000E94793D009741F500D000D0EDB7FEB7B2
:1060D0003196045F1F4FADB7BEB711960D931C9359
:1060E00012978BE59AE282839383CE010196848393
:1060F00095830E94FD3D2DB73EB72A5F3F4F2DBFD0
:106100003EBF892B21F089819A810E94A21DC7017F
:106110000E94442F9C012FC0C80168E67AE20E94C9
:10612000693D0097A1F3C80164E77AE20E94693DE6
:10613000009781F4C7016FEC7DE00E94312F9C0134
:1061400097FD19C0C7016AEE78E045EE54E00E9461
:10615000E12E0BC0E114F10419F42FEF3FEF0BC057
:10616000C7016BE07EE00E94312F9C0118161906D2
:1061700014F420E030E0C9010F900F90CF91DF912F
:106180001F910F91FF90EF900895CF93DF93EC0153
:106190008E819F81009731F00E949E3A1E821F825D
:1061A000188619868A819B81009721F00E94200F12
:1061B0001A821B82DF91CF910895CF93DF93EC0178
:1061C0000E94C53088819981009711F00E94200FAC
:1061D000CE010E949E3ADF91CF910895EF92FF92F7
:1061E0000F931F93CF93DF937C0181E090E06AE0EF
:1061F00070E00E94D539EC018C01009739F180E004
:1062000090E060E070E00E945B108883998397FDC6
:1062100012C06EE97BE2A7010E94200D892B59F480
:106220008881998161E070E04EE251E39E010E9415
:10623000E10C892B59F088819981009711F00E9417
:10624000200FCE010E949E3A00E010E0C801DF91CD
:10625000CF911F910F91FF90EF900895CF93DF930F
:10626000EC018A819B81892B19F0CE010E94C530F7
:106270008881998163EE71E348E451E39E010E94B5
:10628000E00F97FD02C08A839B83DF91CF91089531
:10629000CF92DF92EF92FF920F931F93CF93DF93F2
:1062A0008B01EA017C014115510519F40E94C530AA
:1062B00081C0CA010E94F139D82EC92EC8016D2DA6
:1062C0007C2DAE010E94250C97FD6BC0F701C085A7
:1062D000D185C80FD91FF2E0C130DF0710F0C0E050
:1062E000D2E0F70186819781BE010E94F63A9C01B7
:1062F000F7018683978380859185280F391FFE01DA
:10630000E81BF90BC9016D2D7C2DAF010E944E3D9C
:10631000F701C087D187468157818EE79AE260E016
:1063200070E09E0101E010E00E94012EFC01009748
:1063300079F11082F701C681D781CE0161E87AE256
:1063400044E050E00E94793D009741F5249601C059
:1063500021968881992787FD90950E94273D892B5A
:10636000B9F71C2F0D2F01C021968881992787FD31
:1063700090950E94273D892BB9F31882F70162811D
:106380007381812F902F0E944230892B39F40EC0E7
:10639000F701808591858050924019F4C7010E94D1
:1063A000C5308D2D9C2D0E949E3A04C0C7010E94CD
:1063B000C530EECFDF91CF911F910F91FF90EF90FD
:1063C000DF90CF900895DF93CF9300D00F92CDB799
:1063D000DEB7452B39F0CB01BE016F5F7F4F0E94C6
:1063E000AA0B02C00E94C5302496CDBFDEBFCF915C
:1063F000DF9108951BBEFC0128ED24BF6083089542
:10640000682F772767FD709580EA98E00E94B71C97
:106410000895CF92DF92EF92FF920F931F93CF9345
:10642000DF930E94B01D8AE090E06CEB73E30E9462
:106430009F1D0E94F6338AE090E00E94111C97FD98
:1064400007C180EA98E040E855E260E070E028E0AB
:1064500030E000E010E0A1E0EA2EF12CCC24DD24B5
:106460000E94311C97FDF4C080EA99E040E051EEB3
:1064700060E070E028E030E00E94311C97FDE8C049
:1064800080E090E067EB7CE140EA58E020E030E01B
:106490000E941216EC01009709F4DAC080ED97E033
:1064A00020E233E0F9013197F1F70197D9F760E085
:1064B00072EC81E090E040E02AE73DE10EEC1CE167
:1064C000F0EAEF2EF9E0FF2E0E946D1197FDC0C09B
:1064D00080EA99E040E052EC61E070E028E030E0D2
:1064E00000E010E0E1E0EE2EF12CCC24DD240E944F
:1064F000311C97FDADC088EE93E020E233E0F90156
:106500003197F1F70197D9F783E393E3BE010E9436
:10651000C5098CE493E3BE010E94CE09CE016AEE68
:106520007AE240E050E00E946514CE0164EF7AE226
:1065300040E050E00E946514CE016EEF7AE240E048
:1065400050E00E946514CE0168E07BE240E050E03C
:106550000E946514CE0162E17BE240E050E00E94BF
:106560006514CE016CE17BE240E050E00E946514CE
:10657000CE0166E27BE240E050E00E946514CE016D
:1065800060E37BE240E050E00E946514CE016AE8DF
:106590007BE240E050E00E946514CE016AE37BE2BA
:1065A00040E050E00E946514CE0164E47BE240E0EC
:1065B00050E00E946514CE016EE47BE240E050E0C2
:1065C0000E946514CE0168E57BE240E050E00E9445
:1065D0006514CE0162E67BE240E050E00E94651463
:1065E000CE016CE67BE240E050E00E946514CE01F3
:1065F00066E77BE240E050E00E946514CE0160E86F
:106600007BE240E050E00E946514CE0164E97BE249
:1066100040E050E00E946514CE0160EE7AE240E076
:1066200050E00E94651480EA98E00E94071D892BC3
:1066300051F080EA98E060E070E00E945E1D682FF3
:10664000CE010E9474170E945C0D0E94BA1AEBCF13
:106650008FEF9FEFDF91CF911F910F91FF90EF9000
:10666000DF90CF90089500D000D0EDB7FEB73196FF
:10667000ADB7BEB711968D939C93129786E89AE2B8
:1066800082839383648375830E948B158DB79EB735
:1066900006968DBF9EBF08950F931F93182F092F45
:1066A0006115710571F500D00F92EDB7FEB7319607
:1066B000ADB7BEB711968C93918388E99AE2828335
:1066C00093830E948B158091F82B9091F92B0F905A
:1066D0000F900F900F90009709F44BC00E94DD308F
:1066E0001092F82B1092F92B00D00F92EDB7FEB755
:1066F0003196ADB7BEB711961C9301838AEA9AE230
:1067000030C0CB010E94FD1300D000D0EDB7FEB722
:106710003196ADB7BEB711961C9301832AEB3AE2CE
:1067200022833383848395830E948B158DB79EB714
:1067300006968DBF9EBF80E590E00E94EE3080936C
:10674000F82B9093F92B892BA1F000D00F92EDB785
:10675000FEB73196ADB7BEB711961C9301838AEC94
:106760009AE2828393830E948B150F900F900F9073
:106770000F901F910F9108950E945F1A0895209124
:10678000FC2B3091FD2B21513140C9010895FF921E
:106790000F931F938C01F62E60E070E0CB01BA01DD
:1067A00026E631E040E050E00E9461392091FA2B6A
:1067B0003091FB2B40E050E00E94B3392093FC2B3A
:1067C0003093FD2B3FB7F894F801208181E090E0F1
:1067D00002C0880F991FFA94E2F7880F880F822B66
:1067E00080833FBF1F910F91FF9008950F931F93D8
:1067F000DF93CF93CDB7DEB72A97CDBFDEBFFE01C3
:10680000349687E0DF011D928A95E9F78E010F5FCC
:106810001F4F83E0D8011D928A95E9F72D819E8153
:106820009F7C86E08887217E2D831F8291609E83D6
:1068300080E092E0BF010E94213980E092E067ECA5
:1068400073E30E94F03719821A828B81807F816006
:106850008B8380E092E060E0A8010E94853882E0AE
:106860006FE20E945434182F00E082E06EE20E9432
:10687000543490E0082B192B0093FA2B1093FB2B28
:1068800080E092E00E9425389FB7F894E0E0F2E0C3
:106890008081846080839FBF2A96CDBFDEBFCF9169
:1068A000DF911F910F9108954091CA01E62FFF27B4
:1068B0008093CA0184914093CA010895282F909132
:1068C000CA01E0ECF1E08091CF0187FDFACF83E3CC
:1068D0008287128211822093C00164839287089577
:1068E000DC012091CA01E0ECF1E08091CF0187FD4D
:1068F000FACF83E382871282118290E09093C001E5
:106900008D9184839F5F9032C9F7E0ECF1E022879C
:1069100008951F93CF93DF93C0ECD1E08091CF0116
:1069200087FDFACF1091CA0180E38A878BEC91E052
:1069300061E00E94FA311A87DF91CF911F9108958B
:106940001F93CF93DF93982FC0ECD1E08091CF01BC
:1069500087FDFACF892F90E025E0880F991F2A95AF
:10696000E1F71A8299838093C0011091CA0182E3F2
:106970008A878BEC91E061E00E94FA311A87DF91FF
:10698000CF911F9108951F93CF93DF93982FC0EC61
:10699000D1E08091CF0187FDFACF892F90E035E0DB
:1069A000880F991F3A95E1F71A8299838093C00165
:1069B0001091CA0184E38A878BEC91E061E00E9428
:1069C000FA311A87DF91CF911F9108951F93CF93CA
:1069D000DF93982FC0ECD1E08091CF0187FDFACFF3
:1069E000892F90E045E0880F991F4A95E1F71A82B8
:1069F00099838093C0011091CA0185E38A878BEC4B
:106A000091E061E00E94FA311A87DF91CF911F91E6
:106A100008951F93CF93DF93982FC0ECD1E080911E
:106A2000CF0187FDFACF262F30E02F713070892FEC
:106A300090E055E0880F991F5A95E1F7282B392BE4
:106A40001A8239832093C0011091CA0186E08A8797
:106A50008BEC91E061E00E94FA311A878091C401C9
:106A6000DF91CF911F9108958091CF0187FDFCCFD9
:106A70008091CF0181FF09C086E3E0ECF1E08287DD
:106A80008BEC91E061E00E94FA310895EF92FF9261
:106A90000F931F93E82E00EC11E0F090CA010E94C2
:106AA000343583E3F80182871282118280E080937B
:106AB000C001E4828F5F8032D1F7E0ECF1E0F28632
:106AC0001F910F91FF90EF9008958FEF0E94463530
:106AD0000E94893408951F93182F8FEF0E94463526
:106AE000812F0E94A0341F910895AF92BF92CF9240
:106AF000DF92EF92FF920F931F93C82E062FB42EB2
:106B000070ECE72E71E0F72EF701A2840E94343575
:106B100083E3F701828710E00F711070DD2465E0D8
:106B2000CC0CDD1C6A95E1F70C291D29128211831A
:106B30000083B48285E382878BEC91E061E00E9460
:106B4000FA31F701A2861F910F91FF90EF90DF902D
:106B5000CF90BF90AF9008950F931F938C0182E068
:106B600068E00E945434F801808382E069E00E946A
:106B70005434F801818382E06AE00E945434F801C1
:106B8000828382E06BE00E945434F801838382E0C8
:106B90006CE00E945434F801848382E06DE00E942E
:106BA0005434F801858382E060E10E945434F80196
:106BB000868382E062E10E945434F801878382E098
:106BC00063E10E945434F801808782E064E10E940E
:106BD0005434F801818782E065E10E945434F80161
:106BE00082871F910F9108951F920F920FB60F92F7
:106BF00008B60F9218BE09B60F9219BE0BB60F92C7
:106C00001BBE11242F933F934F935F936F937F93FA
:106C10008F939F93AF93BF93EF93FF93E0E2F2E0E4
:106C200044815581E091FF2BF091002C80E092E0AF
:106C300060E01995FF91EF91BF91AF919F918F9176
:106C40007F916F915F914F913F912F910F900BBE6C
:106C50000F9009BE0F9008BE0F900FBE0F901F90AF
:106C600018951F920F920FB60F9208B60F9218BE8A
:106C700009B60F9219BE0BB60F921BBE11242F93AB
:106C80003F934F935F936F937F938F939F93AF93B4
:106C9000BF93EF93FF93E8E2F2E044815581E091E6
:106CA000FF2BF091002C80E092E061E01995FF91BC
:106CB000EF91BF91AF919F918F917F916F915F9174
:106CC0004F913F912F910F900BBE0F9009BE0F90E7
:106CD00008BE0F900FBE0F901F9018951F920F9235
:106CE0000FB60F9208B60F9218BE09B60F9219BED2
:106CF0000BB60F921BBE11242F933F934F935F93BC
:106D00006F937F938F939F93AF93BF93EF93FF9373
:106D1000E0E3F2E044815581E091FF2BF091002CFB
:106D200080E092E062E01995FF91EF91BF91AF9101
:106D30009F918F917F916F915F914F913F912F9193
:106D40000F900BBE0F9009BE0F9008BE0F900FBEA4
:106D50000F901F9018951F920F920FB60F9208B6C2
:106D60000F9218BE09B60F9219BE0BB60F921BBE3A
:106D700011242F933F934F935F936F937F938F9340
:106D80009F93AF93BF93EF93FF93E8E3F2E04481C7
:106D90005581E091FF2BF091002C80E092E063E0C0
:106DA0001995FF91EF91BF91AF919F918F917F9135
:106DB0006F915F914F913F912F910F900BBE0F906C
:106DC00009BE0F9008BE0F900FBE0F901F90189530
:106DD0001F920F920FB60F9208B60F9218BE09B607
:106DE0000F9219BE0BB60F921BBE11242F933F9327
:106DF0004F935F936F937F938F939F93AF93BF93C3
:106E0000EF93FF93E0E6F2E044815581E091022C9C
:106E1000F091032C80E492E060E01995FF91EF91EE
:106E2000BF91AF919F918F917F916F915F914F91A2
:106E30003F912F910F900BBE0F9009BE0F9008BE8F
:106E40000F900FBE0F901F9018951F920F920FB6C4
:106E50000F9208B60F9218BE09B60F9219BE0BB664
:106E60000F921BBE11242F933F934F935F936F9309
:106E70007F938F939F93AF93BF93EF93FF93E8E636
:106E8000F2E044815581E091022CF091032C80E4E2
:106E900092E061E01995FF91EF91BF91AF919F91C1
:106EA0008F917F916F915F914F913F912F910F90B3
:106EB0000BBE0F9009BE0F9008BE0F900FBE0F9033
:106EC0001F9018951F920F920FB60F9208B60F924F
:106ED00018BE09B60F9219BE0BB60F921BBE112435
:106EE0002F933F934F935F936F937F938F939F93D2
:106EF000AF93BF93EF93FF93E0E7F2E044815581B6
:106F0000E091022CF091032C80E492E062E019956C
:106F1000FF91EF91BF91AF919F918F917F916F9171
:106F20005F914F913F912F910F900BBE0F9009BE33
:106F30000F9008BE0F900FBE0F901F9018951F92D4
:106F40000F920FB60F9208B60F9218BE09B60F92A5
:106F500019BE0BB60F921BBE11242F933F934F9374
:106F60005F936F937F938F939F93AF93BF93EF93B1
:106F7000FF93E8E7F2E044815581E091022CF09123
:106F8000032C80E492E063E01995FF91EF91BF91AB
:106F9000AF919F918F917F916F915F914F913F91B1
:106FA0002F910F900BBE0F9009BE0F9008BE0F904F
:106FB0000FBE0F901F90189522E08030920731F499
:106FC0008091FE2B882359F081E0089580549240EF
:106FD00011F080E008958091012C811181E00895E5
:106FE0002FB7F89432E08030930729F46093FF2B99
:106FF0007093002C07C08054924021F46093022CBF
:107000007093032C2FBF089522E08030920769F41B
:107010008091FE2B8F5F8093FE2B8150A9F481E03D
:1070200090E062E00E94D30708958054924061F49A
:107030008091012C8F5F8093012C815029F482E094
:1070400090E062E00E94D3070895FF920F931F9390
:107050008C01FFB6F8940E940438F80180818160A9
:107060008083FFBE1F910F91FF90089522E0803032
:10707000920769F48091FE2B81508093FE2B882328
:10708000A9F481E090E062E00E94DE070895805458
:10709000924061F48091012C81508093012C8823CF
:1070A00029F482E090E062E00E94DE070895DF921A
:1070B000EF92FF920F931F93CF93DF938C017A018E
:1070C000005E1F4FC62FD0E083E0CC0FDD1F8A95F6
:1070D000E1F7C00FD11F00521040DFB6F894C8018D
:1070E0000E9404388881F70180838A8182838981A4
:1070F0008183C8010E943638DFBEDF91CF911F9196
:107100000F91FF90EF90DF900895DF92EF92FF9242
:107110000F931F93CF93DF938C017A01005E1F4F73
:10712000C62FD0E093E0CC0FDD1F9A95E1F7C00F9A
:10713000D11F00521040DFB6F894C8010E940438F5
:10714000F7018081888382818A8381818983C80154
:107150000E943638DFBEDF91CF911F910F91FF90D3
:10716000EF90DF900895DF92EF92FF920F931F93BD
:107170008C017B01DFB6F8940E940438F80180810D
:10718000807CF7018083F801808D918DF7018583E4
:107190009683F8018281F7018283F8018481F701E7
:1071A0008483F8018381F7018383F8018181F701EA
:1071B0008183C8010E943638DFBE1F910F91FF9076
:1071C000EF90DF9008951F93FC011FB7F894808122
:1071D0008E7F8083CF010E9436381FBF1F91089594
:1071E0000F931F938130910589F08130910528F02C
:1071F0000297A9F020E030E020C082E061E20E9426
:107200005434182F00E082E060E211C082E065E2B1
:107210000E945434182F00E082E064E208C082E04B
:107220006FE20E945434182F00E082E06EE20E9468
:107230005434282F30E0202B312BC9011F910F919E
:107240000895CF92DF92EF92FF921F93CF93DF9337
:10725000EC017B0182E0C030D80719F480E090E0B7
:1072600006C0E2E0C034DE0721F581E090E00E9434
:10727000F0386C011FB7F894CE010E9404382881C1
:1072800082E08883CC86DD86F70185819681888FB0
:10729000998F82818A8384818C8383818B8381818E
:1072A000898321708081282B2883CE010E94363863
:1072B0001FBFDF91CF911F91FF90EF90DF90CF9094
:1072C0000895629FD001739FF001829FE00DF11D30
:1072D000649FE00DF11D929FF00D839FF00D749F50
:1072E000F00D659FF00D9927729FB00DE11DF91FFC
:1072F000639FB00DE11DF91FBD01CF011124089559
:10730000991B79E004C0991F961708F0961B881FF7
:107310007A95C9F780950895AA1BBB1B51E107C058
:10732000AA1FBB1FA617B70710F0A61BB70B881F15
:10733000991F5A95A9F780959095BC01CD010895A4
:1073400097FB092E07260AD077FD04D0E5DF06D08B
:1073500000201AF4709561957F4F0895F6F7909587
:1073600081959F4F0895A1E21A2EAA1BBB1BFD0118
:107370000DC0AA1FBB1FEE1FFF1FA217B307E40714
:10738000F50720F0A21BB30BE40BF50B661F771F6C
:10739000881F991F1A9469F760957095809590954C
:1073A0009B01AC01BD01CF0108950F931F93CF93B3
:1073B000DF93689F8001699F100D789F100D112445
:1073C000C8010E94F139EC01009729F060E070E0FB
:1073D000A8010E94573DCE01DF91CF911F910F91DF
:1073E0000895CF93DF93BC018230910510F462E0E1
:1073F00070E0A091212CB091222CED0140E050E0F2
:10740000E0E0F0E021C0888199818617970769F450
:107410008A819B81309719F08283938304C0809383
:10742000212C9093222CFE0134C06817790738F480
:107430004115510519F08417950708F4AC01FE01B8
:107440008A819B819C01E9012097E9F6411551054C
:10745000A9F1CA01861B970B049708F4BA01E0E072
:10746000F0E02AC08D919C91119784179507F9F44B
:107470006417750781F412968D919C91139730973C
:1074800019F08283938304C08093212C9093222C43
:10749000FD0132964FC0CA01861B970BFD01E80F14
:1074A000F91F6193719302978D939C9343C0FD01E3
:1074B000828193819C01D9011097A1F680911F2CA4
:1074C0009091202C892B41F48091DC2A9091DD2A27
:1074D00080931F2C9093202C4091DE2A5091DF2A1C
:1074E0004115510541F44DB75EB78091DA2A90916C
:1074F000DB2A481B590B20911F2C3091202C24177C
:107500003507B0F4CA01821B930B8617970780F0EA
:10751000AB014E5F5F4F8417950750F0420F531F2A
:1075200040931F2C5093202CF9016193719302C05A
:10753000E0E0F0E0CF01DF91CF910895CF93DF93AA
:10754000009709F450C0EC0122971A821B82A09187
:10755000212CB091222C109709F140E050E0AC179B
:10756000BD0708F1AA83BB83FE0121913191E20F8F
:10757000F31FAE17BF0779F48D919C911197280FD7
:10758000391F2E5F3F4F2883398312968D919C912E
:1075900013978A839B834115510571F4C093212C65
:1075A000D093222C20C012968D919C911397AD01FF
:1075B000009711F0DC01D3CFFA01C283D38321916C
:1075C0003191E20FF31FCE17DF0769F488819981AB
:1075D000280F391F2E5F3F4FFA01208331838A81A4
:1075E0009B8182839383DF91CF9108958F929F92A5
:1075F000AF92BF92CF92DF92EF92FF920F931F93C1
:10760000CF93DF938C01009729F4CB010E94F139CD
:107610008C01BAC09EEFE92E9FEFF92EE00EF11E0D
:107620005801A60EB71EAE14BF0408F4ABC08EEF0F
:10763000882E8FEF982E8A0C9B1CE7014881598178
:1076400046175707B8F04530510508F49DC0CA01E8
:1076500004978617970708F497C042505040461B7E
:10766000570BF4014083518368837983C5010E94DD
:107670009E3A8AC06B01C41AD50AE091212CF09180
:10768000222CC0E0D0E0A0E0B0E042C0E815F9054F
:10769000A1F5208131812C153D0578F1C9010296B3
:1076A0008C159D05A8F04E5F5F4F420F531FE701F9
:1076B0004883598322813381109729F012962D93A4
:1076C0003C93139761C02093212C3093222C5CC0F3
:1076D000225030402C193D0920833183109729F026
:1076E0001296ED93FC93139704C0E093212CF09332
:1076F000222CF7016083718347C080819181C81774
:10770000D90708F4EC01DF01828193819C01F90122
:10771000309709F0BBCF400F511F80911F2C9091E3
:10772000202C84179507E9F4C617D707D0F42091C9
:10773000DE2A3091DF2A2115310541F42DB73EB7FD
:107740008091DA2A9091DB2A281B390BA216B30606
:10775000C8F4A0921F2CB092202CE7016883798393
:1077600013C0CB010E94F139EC01009759F0F701E9
:1077700040815181B8010E944E3DC8010E949E3A4D
:107780008E0102C000E010E0C801DF91CF911F918F
:107790000F91FF90EF90DF90CF90BF90AF909F90B0
:1077A0008F9008952F923F925F926F927F928F9267
:1077B0009F92AF92BF92CF92DF92EF92FF920F9380
:1077C0001F93CF93DF938C011B01EA0161157105B3
:1077D00019F0FB0180839183209749F0CE01029735
:1077E000839728F020E030E040E050E0F6C0F80158
:1077F000A1908F018A2D90E00E94273D892BB9F737
:10780000FDE2AF1631F4F801A1908F015524539495
:1078100007C0FBE2AF1619F4F801A1908F015524BF
:10782000209719F0C031D105C1F4F0E3AF1679F417
:10783000F8018081883711F0883549F4F801A1807A
:107840000E5F1F4FF2E05F2AC0E1D0E006C0209734
:1078500021F480E3A816E9F427C0C830D10531F13E
:10786000C930D10524F4C230D10531F50CC0CA307D
:10787000D10589F0C031D105F9F4C12CD12CE12C0E
:10788000B8E0FB2E28C0C12CD12CE12CA0E4FA2EAC
:1078900022C0CAE0D0E0FCECCF2EFCECDF2EFCECEA
:1078A000EF2EFCE0FF2E17C0C8E0D0E0C12CD12C99
:1078B000E12CE0E1FE2E0FC09E01442737FD4095EC
:1078C000542F60E070E080E090E80E94B339C90175
:1078D000DA016C017D0120E030E040E050E060E042
:1078E0003E01882477FC8094982C70EDB72EBA0C5A
:1078F000E9E0EB1570F48A2D81548A3118F499EC83
:10790000B92E06C08A2D81568A3150F589EAB82EE3
:10791000BA0C8B2D90E08C179D0714F56F3FE1F0AA
:10792000C216D306E406F506B0F0CA01B901A401F7
:1079300093010E9461399B01AC012B0D311D411D4A
:10794000511D2130F0E03F07F0E04F07F0E85F07FE
:1079500010F461E001C06FEFF801A1908F01C5CF75
:107960002114310481F0662331F001501040F101FF
:107970000083118308C051FE1AC002501040F1016B
:107980000083118314C067FF12C050FC05C02FEFA5
:107990003FEF4FEF5FE704C020E030E040E050E809
:1079A00082E290E08093232C9093242C16C050FE0A
:1079B00008C050954095309521953F4F4F4F5F4FF0
:1079C0000CC057FF0AC082E290E08093232C909372
:1079D000242C2FEF3FEF4FEF5FE7B901CA01DF9192
:1079E000CF911F910F91FF90EF90DF90CF90BF90BC
:1079F000AF909F908F907F906F905F903F902F906F
:107A00000895FC0188279927E89421912032E9F311
:107A1000293010F02E30C8F32B3241F02D3239F4DA
:107A2000689404C00E94BD3D820F911D2191205396
:107A30002A30C0F31EF4909581959F4F08958032AF
:107A400009F09111F4C580528F55E0F70895911116
:107A5000EEC5803219F089508550D0F70895911104
:107A6000089581548A5108F4805E855A0895FB0177
:107A7000DC0102C005900D9241505040D8F70895A6
:107A8000FC0105900020E9F7809590958E0F9F1FCF
:107A900008954EED5BE20E94963D0895FB01DC01E6
:107AA00002C001900D9241505040D8F70895DC017A
:107AB00001C06D9341505040E0F70895FB01DC0197
:107AC0000D900020E9F7119701900D920020E1F749
:107AD0000895FB01DC018D91019080190110D9F30B
:107AE000990B0895FB01DC0101900D920020E1F754
:107AF0000895FB01DC014150504030F08D91019020
:107B0000801919F40020B9F7881B990B0895FB011F
:107B1000DC014150504048F001900D920020C9F71F
:107B200001C01D9241505040E0F70895FA01A19123
:107B3000B081009719F41097E1F0CD01DC01CD017F
:107B40000D90002011F4C00113C0FB0121912223EC
:107B500019F02015D9F7F3CFFB012191201519F465
:107B60001E92119606C02223C1F70D900020A1F7A6
:107B7000D001FA01A193B08308957AE0979F902DE8
:107B8000879F802D910D112408950F931F93DF93EC
:107B9000CF93CDB7DEB72E97CDBFDEBF0E891F893D
:107BA000888D998D97FF02C080E090E801978D83C2
:107BB0009E8309831A8386E08C839E01245E3F4F57
:107BC000CE0101966A8D7B8DA9010E944B3E4D81AD
:107BD0005E8157FD0AC02F813885421753070CF488
:107BE0009A01020F131FF80110822E96CDBFDEBF3F
:107BF000CF91DF911F910F910895DF93CF93CDB770
:107C0000DEB72E97CDBFDEBF85E08C838C899D8942
:107C100089839A839E01285E3F4FCE0101966E892B
:107C20007F89A9010E94F4412E96CDBFDEBFCF917E
:107C3000DF9108950F931F93DF93CF93CDB7DEB7F6
:107C40002E97CDBFDEBF8C0177FF02C060E070E8E9
:107C5000615070406D837E8309831A8386E08C8334
:107C6000CE010196BA01A9010E944B3E2D813E81B1
:107C700037FD09C0EF81F8852E173F070CF4F90195
:107C8000E00FF11F10822E96CDBFDEBFCF91DF91A6
:107C90001F910F9108952F923F924F925F926F9292
:107CA0007F928F929F92AF92BF92CF92DF92EF928C
:107CB000FF920F931F93DF93CF93CDB7DEB72B9730
:107CC000CDBFDEBF3C012B015A01FC011682178299
:107CD000838181FD03C06FEF7FEFC6C19AE0892EDB
:107CE0001E010894211C311CF3012381F20123FDA4
:107CF000859123FF81912F01882309F4B2C1853238
:107D000039F423FD859123FF81912F01853229F4D8
:107D100090E0B3010E947D43E7CF982FFF24EE242B
:107D20009924FFE1FF15D0F09B3269F09C3228F4D2
:107D3000903259F0933291F40EC09D3249F0903355
:107D400069F441E024C052E0F52A84E0F82A28C012
:107D500098E0F92A25C0E0E1FE2A22C0F7FC29C0FC
:107D6000892F80538A3070F4F6FE05C0989C902CC1
:107D70001124980E15C0E89CE02C1124E80EF0E2C6
:107D8000FF2A0EC09E3229F4F6FC6BC140E4F42AAF
:107D900007C09C3619F450E8F52A02C0983649F419
:107DA000F20123FD959123FF91912F01992309F071
:107DB000B8CF892F8554833018F08052833038F43F
:107DC00044E050E0A40EB51E5FE359830FC0933624
:107DD00031F0933779F0933509F056C020C0F501A2
:107DE0008081898342E050E0A40EB51E610101E06C
:107DF00010E012C0F501C080D180F6FC03C06FEF27
:107E00007FEF02C0692D70E042E050E0A40EB51E85
:107E1000C6010E9430438C015FE7F52214C0F501D2
:107E2000C080D180F6FC03C06FEF7FEF02C0692DE8
:107E300070E042E050E0A40EB51EC6010E9425434A
:107E40008C0150E8F52AF3FE07C01AC080E290E0EA
:107E5000B3010E947D43EA948E2D90E00817190724
:107E6000A8F30EC0F601F7FC8591F7FE81916F0132
:107E700090E0B3010E947D43E110EA94015010406C
:107E80000115110579F7EAC0943611F0993669F5B4
:107E9000F7FE08C0F501208131814281538184E0E1
:107EA00090E00AC0F501808191819C01442737FD53
:107EB0004095542F82E090E0A80EB91E9FE6F9226B
:107EC00057FF09C050954095309521953F4F4F4F32
:107ED0005F4FE0E8FE2ACA01B901A1012AE030E0C3
:107EE0000E94C343D82ED21840C0953729F41F2DC5
:107EF0001F7E2AE030E01DC01F2D197F9F3661F0E4
:107F0000903720F4983509F0ACC00FC0903739F0A5
:107F1000983709F0A6C004C028E030E00AC010611C
:107F200014FD146020E130E004C014FD166020E16F
:107F300032E017FF08C0F501608171818281938171
:107F400044E050E008C0F50180819181BC0180E0EF
:107F500090E042E050E0A40EB51EA1010E94C34390
:107F6000D82ED2188FE7F82EF122F6FE0BC05EEF66
:107F7000F522D91438F4F4FE07C0F2FC05C08FEEE8
:107F8000F82202C01D2D01C0192DF4FE0DC0FE0106
:107F9000ED0DF11D8081803319F499EEF92208C0AE
:107FA0001F5FF2FE05C003C08F2D867809F01F5FAA
:107FB0000F2DF3FC14C0F0FE0FC01E1510F09D2C09
:107FC0000BC09D2C9E0C911A1E2D06C080E290E0E5
:107FD000B3010E947D431F5F1E15C0F304C01E1530
:107FE00010F4E11A01C0EE2404FF0FC080E390E01A
:107FF000B3010E947D4302FF1DC001FD03C088E75D
:1080000090E00EC088E590E00BC0802F867891F05C
:1080100001FF02C08BE201C080E2F7FC8DE290E03C
:10802000B3010E947D4306C080E390E0B3010E944B
:108030007D439A94D914C0F3DA94F101ED0DF11D4A
:10804000808190E0B3010E947D43DD20A9F706C046
:1080500080E290E0B3010E947D43EA94EE20C1F7F4
:1080600043CEF30166817781CB012B96CDBFDEBF76
:10807000CF91DF911F910F91FF90EF90DF90CF9004
:10808000BF90AF909F908F907F906F905F904F9038
:108090003F902F900895FC0120FD08C023FD05C0EE
:1080A00022FF02C073836283518340830895EF925D
:1080B000FF920F931F9344FF02C033E011C046FFAD
:1080C00002C034E00DC0DB01FC01AA0FBB1FEE1F94
:1080D000FF1F1094D1F76A0F7B1F8E1F9F1F31E087
:1080E000660F771F881F991F3150D1F77B018C01D4
:1080F000E20EF11C011D111DA8019701B701CA0173
:108100001F910F91FF90EF9008950F931F93CF93BE
:10811000DF938C01C8010E943B43EC0197FD08C02E
:108120000E94273D892BB1F7CE01B8010E94A943D7
:10813000CE01DF91CF911F910F910895AF92BF9221
:10814000CF92DF92EF92FF920F931F93CF93DF9323
:10815000EC01C62E5A01122F0E943B43AC018B3218
:1081600019F08D3251F41068CA9409F46DC0CE0133
:108170000E943B43AC0197FD67C06DEFD62ED12224
:108180008D2D807301F54033F1F4CA9409F447C092
:10819000CE010E943B43AC0197FD41C082E0D82A4A
:1081A000483711F0483559F480E4D82ACA94B9F117
:1081B000CE010E943B43AC0199232CF430C0D6FC85
:1081C00002C080E1D82AEE24FF248701242F205307
:1081D000283088F0D4FC09C02A3068F0D6FE05C0EB
:1081E0002F7D822F8151863028F0CA01BE010E9466
:1081F000A94312C02750C801B7014D2D0E94574016
:108200007B018C0182E0D82ACA9461F0CE010E94E1
:108210003B43AC0197FFDACFD1FC04C015C0EE247C
:10822000FF248701D7FE08C010950095F094E094D4
:10823000E11CF11C011D111DC501B801A7012D2D67
:108240000E944B4081E001C080E0DF91CF911F91FF
:108250000F91FF90EF90DF90CF90BF90AF90089577
:108260006F927F928F929F92AF92BF92CF92DF9246
:10827000EF92FF920F931F93DF93CF93CDB7DEB7AB
:10828000A097CDBFDEBF6C01A62E8A017901FE0149
:10829000319680E2DF011D928A95E9F770E030E0C7
:1082A00060E040E050E04F01A1E0B0E0F6018381E2
:1082B000F70183FD259183FF21917F01222309F49A
:1082C0007EC02E3519F44115510569F1872F90E0D4
:1082D0008417950744F42D3551F12D3221F43323C1
:1082E00029F431E021C0332309F4622F322F832F88
:1082F000869586958695F401E80FF11D832F87708A
:108300003D0102C0660C771C8A95E2F72081262980
:108310002083361711F430E007C0361710F43F5FA2
:10832000E6CF3150E4CF71E04F5F5F4FBFCF3323D3
:1083300019F08E8180628E83772359F0FE01319689
:108340009E012F5D3F4F808180958193E217F30757
:10835000D1F7BB24B3944E010894811C911CC60133
:108360000E943B43AC0197FD22C086958695869579
:10837000F401E80FF11D808190E09A0127703070C0
:1083800002C0959587952A95E2F780FD05C0CA0140
:10839000B6010E94A9430BC00115110519F0D801BF
:1083A0004D938D01AA94BB24AA20C9F602C0BB201C
:1083B00031F40115110529F0F801108202C0EE24F4
:1083C000FF24C701A096CDBFDEBFCF91DF911F91E3
:1083D0000F91FF90EF90DF90CF90BF90AF909F9064
:1083E0008F907F906F9008956F927F928F929F925F
:1083F000AF92BF92CF92DF92EF92FF920F931F93B3
:10840000CF93DF935C016B013A01FC011682178266
:108410008824EAC0812F90E00E94273D892B21F01B
:10842000C5010E948540E0C0153249F4F601F3FC15
:108430006591F3FE61916F01653269F415E2C50142
:108440000E943B4397FDDCC0181709F4CDC0B5016D
:108450000E94A943DAC06A3219F0162F00E006C064
:10846000F3FC1591F3FE11916F0101E099240FC007
:108470000260692D70E080E090E040E20E94574089
:10848000962EF601F3FC1591F3FE11916F01212F49
:1084900020532A3068F301FD03C099249A9403C045
:1084A000992009F4B2C0183621F01C3699F4F6016F
:1084B0000BC0F601F3FC6591F3FE6191683619F08B
:1084C0006F01162F07C008600460F3FC1591F3FEDE
:1084D00011916F01112309F498C085E09FE0612F8D
:1084E00070E00E941A43892B09F48FC0802F00FF8F
:1084F00003C0EE24FF2407C0F301E080F18022E0F6
:1085000030E0620E731E1E3651F4F501468157812C
:1085100060E070E0C701202F0E944B4065C0133619
:1085200091F481FD02C099249394C5010E943B43BC
:1085300097FD66C0E114F10419F0F70181937F0102
:108540009A9499F74FC01B3559F4C501692DA701BD
:1085500096010E9430416C01009709F043C03DC074
:10856000C5010E94854097FD4BC01F3659F1103759
:1085700028F4143629F1193639F527C0133719F0C4
:10858000153711F51DC0C5010E943B43EC0197FD55
:1085900011C00E94273D892B29F0CE01B5010E9410
:1085A000A94308C0E114F10419F0F701C1937F0158
:1085B0009A9449F7E114F104A9F0F701108212C06E
:1085C000006203C0006101C00064C501692DA701FC
:1085D000202F0E949E40882329F4F5018381807317
:1085E00079F413C000FF8394F501F380F601F3FCE6
:1085F0001591F3FE11916F01112309F00BCF05C006
:10860000882019F42FEF3FEF02C0282D30E0C90178
:10861000DF91CF911F910F91FF90EF90DF90CF905E
:10862000BF90AF909F908F907F906F900895992703
:1086300088270895FC010590061621F00020D9F73F
:10864000C00108953197CF010895FC010590615054
:1086500070400110D8F7809590958E0F9F1F089558
:10866000FC016150704001900110D8F78095909501
:108670008E0F9F1F0895CF93DF93EC014B8140FF36
:108680001AC046FF0AC04F7B4B838E819F810196A3
:108690008E839F838A81282F2BC042FF13C0E881DD
:1086A000F9818081282F332727FD30952115310549
:1086B00029F440624B832FEF3FEF1BC03196E883D4
:1086C000F98311C0EA85FB85CE0119959C0197FFBE
:1086D0000AC09B812F5F3F4F11F080E201C080E113
:1086E000892B8B83E8CF8E819F8101968E839F8318
:1086F00030E0C901DF91CF9108950F931F93CF937D
:10870000DF938C01EB018B8181FF1BC082FF0DC0C9
:108710002E813F818C819D812817390764F4E8817F
:10872000F9810193E883F98306C0E885F985802FF4
:108730001995892B31F48E819F8101968E839F83B9
:1087400002C00FEF1FEFC801DF91CF911F910F9172
:1087500008959C01FB01838180FF11C086FD0FC03D
:108760009FEF2F3F390759F0228380648F7D8383E9
:108770008681978101978683978330E002C02FEF2F
:108780003FEFC9010895FA01AA27283051F120319D
:1087900081F1E8946F936E7F6E5F7F4F8F4F9F4F95
:1087A000AF4FB1E03ED0B4E03CD0670F781F891FD7
:1087B0009A1FA11D680F791F8A1F911DA11D6A0FA5
:1087C000711D811D911DA11D20D009F468943F9158
:1087D0002AE0269F11243019305D3193DEF6CF0157
:1087E0000895462F4770405D4193B3E00FD0C9F71D
:1087F000F6CF462F4F70405D4A3318F0495D31FD8A
:108800004052419302D0A9F7EACFB4E0A6959795DC
:10881000879577956795BA95C9F7009761057105B2
:1088200008959B01AC010A2E0694579547953795FC
:108830002795BA95C9F7620F731F841F951FA01D56
:068840000895F894FFCF3B
:10884600200000252D3230732025730A0D002400E8
:10885600257320002573202D2068657864756D705A
:10886600286C656E3D2564293A0A00253032782049
:1088760000202020003A200020202025730A00082E
:108886002008000A0D00636F6D6D616E64206E6FC7
:108896007420666F756E643A25730A0D00256300B1
:1088A60068656C70007072696E74207468697320F4
:1088B600696E666F726D6174696F6E002573202D27
:1088C6002068657864756D70286C656E3D25642931
:1088D6003A0A00253032782000202020003A200075
:1088E60020202025730A007375636365737300691E
:1088F6006E76616C696420706172616D6574657213
:108906007300756E6B6E6F776E206661696C75723B
:1089160065006F7574206F66206D656D6F72792FB7
:1089260062756666657273006E6F7420636F6E6E35
:10893600656374656400696E76616C69642073743E
:108946006174650070617273696E67206572726F1B
:10895600720070617468206E6F7420666F756E6445
:1089660000696E636F6D70617469626C65207479FD
:108976007065006E6F207065726D697373696F6ED6
:10898600006F7065726174696F6E206E6F7420730C
:108996007570706F72746564006F7574206F6620F1
:1089A60072616E6765006261642073697A65007240
:1089B60065747279206C61746572006275737900F2
:1089C60064697361626C65640070726F746F636F63
:1089D6006C206572726F720074696D656F757400D4
:1089E60069676E6F7265640063616E63656C65646A
:1089F6002062792072656D6F74650073796E6320ED
:108A06006572726F720061626F7274656400616C88
:108A1600726561647920696E20757365002D2D2D50
:108A260020415353455254494F4E204641494C45E7
:108A360044202D2D2D0A0D002D412D2025733A257C
:108A4600642025733A20300A0D002E2E2F2E2E2F4D
:108A56002E2E2F2E2E2F746F6F6C6B69742F6F77DF
:108A66006C2F636F72652F6F776C5F6572722E6302
:108A760000756E6B6E6F776E002D2D2D2041535352
:108A8600455254494F4E204641494C4544202D2DD0
:108A96002D0A0D002D412D2025733A2564202573BE
:108AA6003A202128746D6F2D3E666C61677320260F
:108AB60020544D4F5F44454C45544544290A0D000A
:108AC6002E2E2F2E2E2F2E2E2F2E2E2F746F6F6CB6
:108AD6006B69742F6F776C2F636F72652F6F776C6E
:108AE6005F74696D65722E630045004E004F004D40
:108AF6000053002D2D2D20415353455254494F4EBE
:108B0600204641494C4544202D2D2D0A0D002D416E
:108B16002D2025733A25642025733A20300A0D004E
:108B26002E2E2F2E2E2F2E2E2F2E2E2F746F6F6C55
:108B36006B69742F6F776C2F706F7274732F6176F9
:108B460072382F6F776C5F756172742E63000065E3
:108B56007272006F6B002573202564202825732907
:108B66000A0D0075736167653A206765745F686F03
:108B7600737462796E616D65203C646E736E616DAF
:108B8600653E0A0D00636F6E6E5F636220736F63EE
:108B96006B69643A256420636F6E6E656374656401
:108BA6003A25640A0D006C6F6F6B75705F63623AED
:108BB60020686F7374206E6F7420666F756E640A1A
:108BC6000D006C6F6F6B75705F63622069703A257C
:108BD600730A0D002573202564202825732920009B
:108BE600706565723A25730A0D0075736167653A9B
:108BF600206765745F7065657261646472203C739A
:108C06006F636B69643E0A0D0073656E64696E6717
:108C160020256420627974657320746F2025733A69
:108C260025640A0D0077726F74653A2564207265B3
:108C36006D61696E3A25640A0D0075736167653A60
:108C46002073656E64746F203C736F636B69643E5A
:108C5600203C69703E203C706F72743E203C64611B
:108C66007461202E2E2E3E0A0D0073656E64696EA9
:108C7600672025642062797465730A0D0075736137
:108C860067653A2073656E64203C736F636B696435
:108C96003E203C64617461202E2E2E3E0A0D007526
:108CA600736167653A20636C6F7365203C736F630D
:108CB6006B69643E0A0D0075736167653A20636FE0
:108CC6006E6E656374203C736F636B69643E203C13
:108CD60069703E203C706F72743E0A0D0028636F07
:108CE6006E6E656374696F6E206C6F737429000015
:108CF60072785F636220736F636B69643A256420E0
:108D06006C656E3A25642025730A0D00525800756D
:108D1600736167653A206C697374656E203C736F86
:108D2600636B69643E205B6261636B6C6F675D0AAF
:108D36000D006C697374656E5F636220736F636B9D
:108D460069643A25642C20616363657074696E6793
:108D5600202E2E2E200075736167653A2062696E9B
:108D660064203C736F636B69643E203C69703E20EF
:108D76003C706F72743E0A0D0073747265616D000B
:108D8600646772616D007261770075736167653A39
:108D960020736F636B6574203C73747265616D7CC0
:108DA600646772616D7C7261773E205B70726F746E
:108DB6006F636F6C5D0A0D0025732025642028659E
:108DC6006E61626C65643A2564290A0D00757361EB
:108DD60067653A207365745F64686370203C307C15
:108DE600313E0A0D00257320256420280069703A5B
:108DF600257320006D61736B3A2573200067773AFF
:108E060025732000646E733A2573290A0D00757365
:108E16006167653A207365745F6970616464722086
:108E26003C69703E205B6D61736B5D205B67775DAF
:108E3600205B646E735D0A0D004E2F410025732082
:108E460025642028257320253032783A253032785B
:108E56003A253032783A253032783A253032783A27
:108E660025303278290A0D0025732025642028250F
:108E76003032783A253032783A253032783A253011
:108E860032783A253032783A25303278290A0D0080
:108E960075736167653A206C696E6B7570205B73DC
:108EA6007369645D205B6B65795D205B7765705DDA
:108EB6000A0D006C696E6B757000776C705F6C697B
:108EC6006E6B757028737369642C206B65792C2022
:108ED60077657029006C696E6B646F776E00776CCE
:108EE600705F6C696E6B646F776E282900676574B6
:108EF6005F68776164647200776C705F6765745F42
:108F06006877616464722829006765745F6E6574AA
:108F1600776F726B00776C705F6765745F6E6574F0
:108F2600776F726B2829007365745F69706164647A
:108F36007200776C705F7365745F697061646472E8
:108F46002869702C206D61736B2C2067772C206448
:108F56006E7329006765745F697061646472007777
:108F66006C705F6765745F6970616464722829005C
:108F76007365745F6468637000776C705F736574A3
:108F86005F6468637028656E61626C652900676559
:108F9600745F6468637000776C705F6765745F64A4
:108FA600686370282900736F636B657400776C7053
:108FB6005F736F636B657428747970652C207072AB
:108FC6006F746F290062696E6400776C705F626906
:108FD6006E6428736F636B2C2069702C20706F721F
:108FE6007429006C697374656E00776C705F6C69C8
:108FF6007374656E28736F636B69642C206261639A
:109006006B6C6F672900636F6E6E65637400776CB7
:10901600705F636F6E6E65637428736F636B6964EC
:109026002C2069702C20706F72742900636C6F732A
:109036006500776C705F636C6F736528736F636B25
:109046006964290073656E6400776C705F73656E82
:109056006428736F636B69642C20646174612900F2
:1090660073656E64746F00776C705F73656E64749D
:109076006F28736F636B69642C20646174612C20A4
:1090860069702C20706F727429006765745F706553
:1090960065726164647200776C705F6765745F7097
:1090A6006565726164647228736F636B6964290015
:1090B6006765745F686F737462796E616D6500775A
:1090C6006C705F6765745F686F737462796E616DEB
:1090D6006528646E736E616D6529000A0D007474EF
:1090E6006370206572723A256420282573290A0D5B
:1090F6000074746370206F6B3A2025642062797463
:1091060065732070726F63657373656420696E2082
:109116002564206D732C2025642E2564204B422F58
:10912600730A0D0074746370206F6B3A20256420F7
:1091360062797465732070726F63657373656420FA
:10914600696E2030206D730A0D002E002D2D2D2006
:10915600415353455254494F4E204641494C45448C
:10916600202D2D2D0A0D002D412D2025733A256425
:109176002025733A20707269762D3E73656E640AF7
:109186000D002E2E2F2E2E2F776C705F7474637049
:109196002E63002D412D2025733A25642025733A30
:1091A60020706F73203D3D20707269762D3E62758A
:1091B600666C656E0A0D002D70002D6E002D6C001C
:1091C6002D74002D7200257320256420282573290F
:1091D6000A00657272007474637020636F6E6E6548
:1091E60063742025733A2564206E6275663A256499
:1091F600206275666C656E3A256420736F636B69D1
:10920600643A25640A0D0074746370206C69737483
:10921600656E20706F72743A2564206275666C659F
:109226006E3A2564206C736F636B69643A25640A31
:109236000D0075736167653A2074746370205B2D49
:109246007472706E6C5D0A0074746370007474637B
:1092560070207468726F75676870757420746573B2
:1092660074004E2F4100253032783A253032783A54
:10927600253032783A253032783A253032783A2518
:109286003032780025642043002F002F3F002F69DD
:109296006E6465782E68746D6C3F00746F67676CDA
:1092A600653D4C45442564002F696E6465782E68DB
:1092B600746D6C002F6C6F676F2E676966000D0A00
:1092C6000047455420006C696E6B5F6362206C69D1
:1092D6006E6B3A25640A0D00616464725F636220F6
:1092E60069703A6E6F6E650A0D006874747064205A
:1092F60073746F707065640A0D00616464725F63F5
:10930600622069703A25730A0D00687474706420CF
:10931600737461727465640A0D002000252C0000C8
:109326006020D415652000000000732683287A2665
:1093360000000000952647289E2600000000AD2666
:10934600FB27B82600000000C9265527D5260000B1
:109356000000E7269826F226000000001427E425E0
:109366001F270000000030276E2539270000000067
:109376004E273125572700000000662785246D27D4
:10938600000000008527D5238A2700000000A327B8
:10939600D222AA2700000000C627B621CE27000049
:1093A6000000EC274021F227000000000428452099
:1093B6000928000000002028141F272800000000AC
:1093C6004A287C1E5728000000007028C61D7F28EA
:1093D60000000000082AA02C0D2A00000000000052
:1093E6000000FFFFFFFF6F776C5F6572726F7200A0
:1093F6006F776C746D725F64656C746D6F006F77F8
:109406006C756172745F70617269747900636F6EF6
:0E9416006E5F63620073656E646275660000CF
:00000001FF
